:020000041100E9
:1030000070B500234025294C0120636101F0F4F9DB
:103010000223FE212800264A257401F073FA0028B5
:1030200035D10223FF21234A207C01F06BFA0028CE
:103030002DD1214BA2899A4226D1E3891F4A93427E
:103040000ED11F4B1F4963612368002B05D1002956
:1030500003D00C22200008F0D7FC01F041FA70BD2B
:10306000194A934201D00021EEE7184B184A1B6819
:10307000934205D9C02204212800920001F0BCFA35
:103080000F4B14496361DFE700232374EBE7CC2285
:103090003820AC219201207401F0AEFA0028F3D15F
:1030A0000D4B0E4963610E4BE381CDE7E862FF1FD4
:1030B000F462FF1FF662FF1F5959000083050000EC
:1030C00079420011BCBB0011821500002C63FF1F68
:1030D00087130000C8BB001101430011B0BB0011F1
:1030E000AAAAFFFFF7B5164B0192C318021D0020D4
:1030F000009388235B05D3181B685C1C1AD09CB214
:10310000402C18D88D781E0CAC466746CD782D0221
:103110003D43AE4206D1019800280ED110000C703C
:10312000240A4C7003249BB20733A343D218009B9C
:103130009A42DED3FEBD4432F9E71000FAE7C046FA
:10314000FC0F0000802213B503000324019189B213
:10315000520107319B18A14304305A1A88235B059A
:10316000C3181B68591C03D190429241104016BDF0
:1031700099B2402907D80B000733A343C0189042E7
:10318000ECD30020F3E74430F9E7134B134A1B68F4
:10319000126810B5FA24934201D81A00F824104B93
:1031A000E4021B689A4210D813000E4A12689A4231
:1031B0000ED3013307D1F823DB029C4203D10A4925
:1031C000054808F081FA200010BDFC24E402ECE779
:1031D000FE24E402F7E7C04600C0071100D0071143
:1031E00000E0071100F00711FFFFFF7FF0B59BB073
:1031F000150004900391402A00D9A0E006AB598045
:103200001A80FFF7C2FF0400042816D9002206A97D
:10321000FFF768FF052810D906AB1B88AB420CD11D
:10322000002D07D0514B2A000499C01808F08CF9E2
:10323000002802D101201BB0F0BD06AB1D8020008C
:103240000699FFF77FFF041E7BD1069B0793FFF7CC
:103250009CFF80235B01C618802307001B039E424E
:1032600001D3F826F60288235B05F31801931B6847
:10327000013302D0019808F057FA3D49019808F04F
:1032800023FA3B1D0293331D05938822029B5205AE
:103290009B181B6808935A1C3CD044219AB2009199
:1032A000402A04D80320D11D814389B2009103999B
:1032B0001B0C8B4224D0402A22D80122300008A9BE
:1032C000FFF710FF021E1BD1380008A9FFF70AFF05
:1032D0000400042831D9009A059B9B1880225201D2
:1032E000B218934240D288235B05C118009A09A8FE
:1032F00008F0A2FA1D4B009A09A9F01808F0ACFBDF
:10330000009A029B9446634402931A4B029AFB185C
:103310009A42BAD388235B05FC18216801980139C9
:1033200008F0D2F9200008F0FFF9039A07AB5A80A1
:1033300030000799FFF706FF0400002C03D100209E
:1033400079E70428FBD988235B05E018069908F083
:10335000BBF90323EA1C9A4300D16BE7034B0499A2
:10336000E01808F079FB65E70424ECE7040000119D
:10337000FFFFFF7FF80F0000F7B505001400402A9B
:1033800021D8002701AE71803780FFF7FEFE0428A8
:1033900016D93A003100FFF7A5FE042810D9368867
:1033A000BC420BD0BD4209D0221CB44200D9321C11
:1033B000064B92B2C118280008F03EFA30B2FEBDAA
:1033C000C04300B2FBE703204042F8E704000011CD
:1033D00037B5042204000D0001A81649FFF7CCFF01
:1033E000020004280BD1019BA34208D3AB4204D0B6
:1033F000104901A80195FFF7F9FE01203EBD0E4CD2
:1034000023682000019308F08FF901992000013909
:10341000019108F059F980235B01E418074B9C42A5
:10342000EED10422034901A80195FFF7DFFE002039
:10343000E4E7C0465555000000C007110000081120
:1034400030B589B008F060F910226946254808F0C7
:103450002BF8254B009A9A420ED1019B029A0F2B12
:1034600033D8002101240698013B08D2002900D05E
:103470000292029B013331D10023029325E0551CB7
:10348000F2D102002100EFE710341022200004A93D
:1034900008F00AF8029B013301D1069B02938823AE
:1034A00004995B05C918059B06981A03120B049131
:1034B0000592814203D02B4201D108F0A5FA019B6D
:1034C000013B0193019B002BDED1029B002B03D01B
:1034D000049304984168084709B030BDE025014CC9
:1034E0002D03EFE70000011150485936F7B50F4999
:1034F0000F4B0A6804001A4084235B0013430B60DF
:10350000030003271033019300252E00112008F03B
:1035100043FA084B1B683B40AB4002351E43202D4D
:10352000F4D1019B40C4A342EED1F7BD5CF0004052
:1035300000FEFEFF64F00040802270B5AD4CAE4B43
:10354000D200002120001C6008F08EF92300AB4A55
:1035500088331A60AA4B1A786E23002A00D01133E0
:10356000E3620A232365A74B1878A74BA0630138B1
:10357000E361C3B2032B01D810232362A34B37228C
:103580006361C823DB00A36123008C331A60082326
:1035900036210F3AE518E16323646264E967043970
:1035A000251DE96725003B26BC352E602500C0356A
:1035B0002B602500C4352A6025000636CC352E60E8
:1035C0002500083EC8352E602500D0352960210031
:1035D000D4310B602100D8310A6021000225E0318E
:1035E0000D6025004221DC35296025001B3EE435B5
:1035F0002E602500E8352B602500EC352A6022007E
:103600000525F43215602200F032116022001831D5
:103610009032116022009432136023003C229833D0
:103620001A60AF23DB002360794B2363032805D89E
:1036300007F0AAFF33023537152363609623210074
:10364000FA225B00A360E360C8332361714BFC3155
:103650009200A3640A6062626F4A704DA262732294
:10366000E2656D3A6265A2650232E5644A60022154
:10367000616696218900A166626709210022E166E0
:10368000A2676749674A684E2167E2673560032889
:1036900011D807F079FF96089EA61023CDE70E23D8
:1036A000CBE70C23C9E720001A259C3005602000D9
:1036B0000735A03005602000A83003602300FA2001
:1036C000F8338000186023006420A43318602300BE
:1036D0005F38AC33186023000338B0331860230020
:1036E000C630B433186023000020B83318602300BC
:1036F0003825FC339D604D4D5A665D644C4D9A648F
:10370000DD619625AD001D624A4D9A675D62F53D0B
:10371000FF3D9D621E25484ADD6618675867D965DA
:103720001966DA67BE23C021444A5B00E250444B6D
:103730004900635004316250C4225200A350FA235E
:10374000E4205B000432A3500432A3503D493E4ABA
:103750003E4BD1603E49800019503E49E938FF3860
:1037600019503D49043019503C491038D1613C4949
:1037700011633C4951633C4911603C49195019009F
:103780003B48F83108603B49D16582213A4A8900BB
:103790005A501A0039490832D1671A003849B432F0
:1037A00011608821374A89005A501A0036498832F8
:1037B0001160364ADA6408F06FF9012008F0ACF8BD
:1037C00070BD200014259C30056020000435A03019
:1037D00070E7200010259C30056020000335A030E4
:1037E00068E720000E259C30056020000235A030DF
:1037F00060E7C0460004FF1FC465FF1FB070FF1FD5
:103800007C45FF1F4A0AFF1F3A07000080C3C90119
:103810009A02000050C300006A180000280A000045
:10382000204E000088130000F009FF1F0040001127
:1038300068100000C4090000DC05000040420F00D1
:1038400010270000FD1BFF1FFC00FF1F0000FF1FD3
:10385000252FFF1F4D32FF1FE530FF1FD91FFF1F10
:10386000F51FFF1FA121FF1F491FFF1FC528FF1FB5
:103870008D2CFF1FD918FF1FD127FF1F3925FF1FD0
:103880004525FF1F491EFF1F011FFF1FC11DFF1FF1
:10389000F7B50B0CFF270122009300233C001E000C
:1038A0001D009446019089B262469A40100008407B
:1038B00018413618B6B2FF2F02D1012E00D19FB2A7
:1038C000009802401A41AD18ADB2FF2C02D1012D73
:1038D00000D19CB20133102BE6D10320012E07D179
:1038E000012D04D1019B2401E4191C700138FEBD97
:1038F000102EFCD10238102DF9D00230F7E710B5A8
:10390000064C2378002B07D10548FFF7EFFD05484B
:10391000FFF7ECFD0123237010BDC0468465FF1F37
:103920009865FF1F8865FF1FF0B58BB00D00012360
:103930000190102936D8FFF7E2FF00231A001B4838
:10394000C15C01335218102BFAD1023B002A29D056
:10395000174B184C1F68002306A9E25C1600FA5C9E
:1039600056405E540133102BF7D102AA07F064FED3
:103970002A0002A9019808F047F807F055FE2368CD
:103980001B18236007F050FE63681B18636007F084
:103990004BFEA3681B18A36007F046FEE3681B18E4
:1039A000E360002318000BB0F0BDC0469865FF1F10
:1039B0001C44FF1F8865FF1F0223F0B50124574EEA
:1039C000574D3370574B2C701B688FB0552B10D050
:1039D000082006F0F5FA00280BD000232100009300
:1039E0000420514A07F058FF8023DB059C62FFF753
:1039F00027FD002006F07CFD07F096FDFFF79CFDFB
:103A000007F062FF1F2201240021484B0EAF1A70FD
:103A1000474B1C70474B1970474B19689143163A36
:103A20000A431A60602219689143403A0A431A60B7
:103A300007F002FD07F018FEC120FF213F4B800078
:103A40001A588A431A50C522920098588843BF39A1
:103A50000143995098583A4908408021C9010143CF
:103A6000802099509958C0050902090A01439950CC
:103A700080213448490107F00FFD03232200324919
:103A800001940093314807F0C7FF2C22304903A866
:103A900007F0D2FE03AC61782078023406F0B6FA63
:103AA000BC42F8D10121002006F0CAFB294B2A4A6A
:103AB000196803201140A022D2020A431A60802212
:103AC000196892040A431A601968244A1140802236
:103AD00092030A431A60224B224A934200D80120E3
:103AE00007F0E2FF07F0B8FD07F0EEFF307807F0CF
:103AF0007BFF2878C0B207F097FE07F015FF0A4950
:103B0000042007F0D1FE06F0BFFC00F09FF800F0A3
:103B100031FE00F00BFA00200FB0F0BD4A0AFF1F83
:103B20007C45FF1F34F000403B000108480AFF1F9E
:103B3000490AFF1F680AFF1FBCF0004000E100E0D7
:103B4000FF00FFFF8045FF1F0458FF1F8055FF1F28
:103B5000D8BA001114F00040FF7FF8FFFFFF9FFF6D
:103B6000B070FF1F0080FF1F70B500252849294A4B
:103B700029484D6308CA1B051B0DED188242F9D177
:103B80000022264B8B63264B08211A628022254B8C
:103B90009205DA67244BDA688A43DA60234A12789E
:103BA000012A03D09A6822490A409A600121EE2432
:103BB0002048E40002686C438A430260DA681120FE
:103BC0008A43DA6007F0F8FC112007F0A5FC112009
:103BD00007F09AFE184A200C0400642390420AD889
:103BE000FA220023D200904205D9144B0A21C018B2
:103BF00007F0BAFEC3B2124A1372124BD4801B787C
:103C0000002B04D1104B1021187807F065FD70BD12
:103C1000000005408805054000060540FF01000042
:103C200000F0004004E100E03CF000404A0AFF1FC1
:103C3000FFDFFFFF00380040B70B000030F8FFFF48
:103C40000063FF1F3865FF1F2863FF1F002210B5A8
:103C50001100112007F048FE10BD0000F8B5002348
:103C600001250826394F3A4C3B62E3681120AB43EB
:103C7000E360E368B343E36007F04EFC112007F014
:103C80009BFC112007F098FD402322682900134374
:103C9000236080236268DB02134380226360A36891
:103CA00007201343A360A3682A4A1340A36080231C
:103CB000A2689B0113431022A360236C93432364E7
:103CC000236C2B43236480235B003B62226B224BDB
:103CD0001A402263626B1A406263A26B1A40A263AD
:103CE000E26B1340E3631D4AE3681340E36006F0B0
:103CF00077FA2900072006F0A3FA8021184A11203C
:103D0000536C0B43536407F087FDFD21154B164A96
:103D100089005A508023C720626B5B03134363639F
:103D2000E36880003343E360E368104A1D43104BAF
:103D3000E56019581140802212020A431A5080226D
:103D400092051A600B4B5E63F8BDC04600F0004060
:103D50003CF00040FFFFDFFFEFFFEFFFFFFF7FFFC3
:103D6000003800400000FF1F693B0011FF00FFFF0B
:103D700000E100E00000054030B503A804880B20F6
:103D8000002C0ED14968074D087849780902014393
:103D90000A20A94205D1012120001980024B1B7A7B
:103DA000137030BD192A00000063FF1FF7B515001E
:103DB00008AA16884A680F4F1478527812022243D4
:103DC0000A24BA4214D10122DBB2019200962A00E1
:103DD00007F0AAFA041E0BD1074B1B68002B07D073
:103DE00068782A78000210434242504101309847D7
:103DF0002000FEBD022900008462FF1F30B50125AE
:103E000003790400BFB02B4212D00A49408806F063
:103E1000F7FD28420CD06A46074B69465B8D5580FA
:103E20001380064B60881B7A1371002203F0AEFEEC
:103E30003FB030BD7C62FF1FC041FF1F0063FF1F0A
:103E400010B50549054806F091FD0421044A0548CE
:103E500006F04EFD10BDC0467C62FF1FFFFF000054
:103E600004BB0011C041FF1F10B5024804F010FD53
:103E700010BDC046FD3D0011062383701033037151
:103E8000443B43712A3383714433C37100230222BC
:103E9000012110B503720E4B027041701C888172B3
:103EA0004472197A0273C1729A784273DA78827313
:103EB0000322C2731A7902745A7942740C228274F2
:103EC0009A79C274DB7903751123C37010BDC046A3
:103ED0000063FF1F10B5142007F06EFD124B142273
:103EE0000021186007F0C8FD002007F035FC012014
:103EF00007F0DAFB022007F097FD032003F06CFFC8
:103F0000042005F081FF052003F0AAF9062003F044
:103F100077FE072001F0D2F8082006F0C9FC09203E
:103F200000F0A8FE10BDC0468862FF1F10B507F064
:103F300053FB012007F0F0FB07F026FD002010BD29
:103F4000094B10B50400984205D0012904D1200086
:103F5000064906F00BFD10BD0229FCD1013904F021
:103F600055FC0028F3D0F6E7FEFF0000AE62FF1F0D
:103F700070B50D7A100004AA2C0016881022144087
:103F8000154220D1002E20D10A78022A18D14A6881
:103F9000517815780E4A09022943914205D00D4AFD
:103FA000914209D01C800A2404E014220A491A8094
:103FB00007F02AFD200070BD0C2208491A80F7E79F
:103FC0001C800124F6E70824F4E70B24F2E7C0463E
:103FD000F3FF0000F4FF00000044FF1FE0BB0011EE
:103FE00010B504000749084806F0C0FC074804F073
:103FF0008FFB0020E40704D50721054A054806F099
:1040000077FC10BDAE62FF1FFFFF0000413F0011B3
:1040100048BB00110442FF1F00B50C4BBFB01A781B
:104020000B4901A800F0DAFB6B4680B258800028EB
:1040300009D06A46074B69461B881380064B00224D
:10404000188803F0A3FD3FB000BDC0468C62FF1F7F
:104050008D62FF1F5E42FF1F5E43FF1F00B50C4BCA
:10406000BFB01A780B4901A801F0D2FC6B4680B2B0
:104070005880002809D06A46074B69465B8D13803B
:10408000064B0022188803F081FD3FB000BDC046FA
:10409000B662FF1FB762FF1F0442FF1F5E43FF1F90
:1040A000F7B50E00377A1C0008AB11003D001A88E6
:1040B00020231D401F423CD13378022B3BD1736833
:1040C0001F785B781B023B431E4FBB4208D01E4F3C
:1040D000BB4214D01D4DAB4221D00A252800FEBDA5
:1040E000002A2AD1142C2AD82200F06807F08CFC70
:1040F000174B1C70012CF1D9FFF7B0FFEEE7002A37
:104100001BD1202C1BD82200F06807F07DFC114B3E
:1041100004211C70104B187807F0DEFADEE7E3B2DA
:104120000124009201940A00310007F0FDF8050017
:10413000D4E70825D2E70125D0E70B25CEE70D25EA
:10414000CCE7C046F3FF0000F4FF000002290000A6
:10415000B662FF1F8C62FF1F2863FF1F07B5074B66
:1041600001A9188803F0FEFC172805D1044B1E2274
:104170004021187807F0B0FB07BDC0465E43FF1F23
:104180002863FF1F70B5160004AA148805AA1578C5
:104190004A685078117800022A4A08438018052896
:1041A0004BD807F0F1F903131E29343F0720032CE5
:1041B0000BD80422121BAA4200D92A0022491A80D5
:1041C0003000091907F020FC002070BD0720112CD9
:1041D000FBD81222121BAA4200D92A001B491A80BE
:1041E000EEE707200E2CF0D80F22121BAA4200D9AE
:1041F0002A0017491A80E3E70720032CE5D8042298
:10420000121BAA4200D92A0012491A80D8E70720B7
:10421000032CDAD80422121BAA4200D92A000E4924
:104220001A80CDE70720032CCFD80422121BAA4204
:1042300000D92A0009491A80C2E700220A201A8000
:10424000C3E7C046DCD5FFFF93BB0011D462FF1F5C
:1042500083BB00117EBB001179BB001174BB001140
:1042600010B50D21024A034806F042FB10BDC046BE
:1042700068BB00117442FF1F37B5012000F0BCF885
:104280001C4D0223002101AA287C00F03BF96A465C
:10429000040002230121287C063200F033F9044394
:1042A00000F01EF9002C22D16B469A882B68D2BAF6
:1042B00053432A8910491B149B184B806B46DA889C
:1042C0006B6852BA5204520C53436A891B0C9B18F8
:1042D0000A481A1C1BB2834200DD021C130400D5DD
:1042E00000220B888A8001330B8020003EBD012410
:1042F000FBE7C046E862FF1F0063FF1F0F270000B7
:1043000037B5012000F078F81E4D07226946287C59
:1043100000F026F9041E31D16B461B787F2B2DD877
:1043200000F0DEF86B46D878F02302041B031A4035
:104330006B469B8814495BBA9BB21A432B680009F1
:1043400053432A891B0C9B184B806B465A789B78E9
:1043500012031B011A436B68024353436A891B0C07
:104360009B181AB21B0402D58C8020003EBD074B5F
:104370009A4201DC8A80F8E78B80F6E700F0B0F81B
:104380000124F2E7E862FF1F0063FF1F0F27000010
:1043900010B50E4C237C002B0CD0382B0BD10120F8
:1043A00000F02AF8CC22AC21207C920100F024F904
:1043B00000F096F810BD402BFCD1012000F01CF855
:1043C0000021207C00F0F8F8F2E7C046E862FF1F09
:1043D00010B5084B1A7C002A09D05B69002B06D067
:1043E0009847041E01D0FEF70BFE200010BD0124EB
:1043F000F9E7C046E862FF1F70B5002106001620ED
:1044000005F05AFF0121152005F056FF07F064F86A
:104410000400092007F0D0F900222B4B2B4DDA665F
:1044200061321A6019685B3A9143002E28D0023A33
:104430000A431A60AC4209D10A22DA6107321A62D1
:1044400000221A639A630132DA6370BD204A9442F3
:1044500003D11E22DA610532F1E71E4A944203D1EC
:104460003022DA610632EAE71B4A944203D1432242
:10447000DA610832E3E7194A9442E1D16922F7E7A9
:1044800002220A431A604622AC4203D0104A9442E8
:1044900004D194225A6106329A61D1E70D4A9442BE
:1044A00001D1E622F6E70C4A944204D13422FF32CD
:1044B0005A610D32F0E7094A9442C1D1E622520016
:1044C0005A610A32E8E7C046005000400024F40078
:1044D0000048E801006CDC020090D00300D8B80569
:1044E00010B50024064B0920DC6607F015F8210002
:1044F000162005F075FE2100152005F071FE10BD97
:1045000000500040F8B51C000023134D0F00EB666F
:104510006860160007F0F8F801238022EB6623009C
:104520002F615200013B08D206F0DEFF08200B4A43
:104530001168002C03D12000F8BD2A61F2E72B6F2F
:10454000034203D02B69013C3370013613685B1AB8
:10455000012BEED90124EEE7005000406008FF1F58
:10456000002370B5124D1400EB6668600E0007F072
:10457000CBF801238022EB6623005200013B08D2D6
:1045800006F0B2FF08200B4A1168002C03D120006E
:1045900070BD2A61F2E72B6F034203D02B69013C07
:1045A0003370013613685B1A012BEED90124EEE754
:1045B000005000406008FF1F002370B50C4C0D0038
:1045C000E366606007F0A0F80123E366256106F06A
:1045D0008BFF8020074A80001168636B034205D17E
:1045E00013685B1A012BF8D9012070BD0020FCE78D
:1045F000005000406008FF1F002370B5134C0E00F0
:10460000E3666060150007F07FF80123E36626612A
:104610000F33626B1A42FCD02B0A23611023626BAA
:104620001A42FCD0EDB2256106F05EFF8020084AF8
:1046300080001168636B034205D113685B1A012B7C
:10464000F8D9012070BD0020FCE7C04600500040B2
:104650006008FF1F002370B5124D0C00EB66686008
:10466000160007F051F80123A619EB660F33B44288
:104670000ED106F039FF80200B4A800011686B6B69
:1046800003420CD113685B1A012BF8D9012070BDCD
:1046900022782A616A6B1A42FCD00134E7E70020D5
:1046A000F5E7C046005000406008FF1F0A4B0B4A68
:1046B00019689068884202D980235B04C91853683E
:1046C00091601B1A5B181168D80B5B0440185B0CD7
:1046D000106053607047C04628F000401863FF1F09
:1046E00010B51B4B1A793F2A01D93F221A7119794B
:1046F000184A1948117018221849028018480A806F
:1047000002804A809A791748802402800C208A808F
:10471000013242432401101CA24200D9201C124A3B
:10472000C88010805A79002A01D101325A711A7A50
:10473000012A01D802221A725A791B7A0B48534374
:104740000A21584307F010F9094C206010BDC046FB
:104750000C63FF1F480AFF1F5C43FF1F2845FF1F14
:104760005A43FF1F0465FF1F5843FF1F71020000DB
:104770002C63FF1F10B507210020FEF729FE124C05
:10478000002807D10C222000104907F03DF9FFF75F
:10479000A7FF10BD0C2220000D49FEF7EDFD0C28EF
:1047A00004D00C222000094907F02EF9094C0C22F4
:1047B00020000949FEF7E0FD0C28E8D00C2200217A
:1047C000200007F059F9E2E70C63FF1FD4BB00118A
:1047D000FC0C0000E862FF1FF50C0000F0B50400BF
:1047E0000E00150085B0002A00D1BBE0087800213A
:1047F00020706170262800D184E00FD8072805D8E2
:1048000006F0C2FE5A3535353588968F232800D1FB
:10481000BFE025285ED0FF23637098E0712800D1A7
:104820008DE01ED8562851D0602800D19CE0552834
:10483000F1D1013A874D0C2A46D8002A0AD0711CC2
:10484000280007F0E1F8FFF74BFF0C22280082490F
:10485000FEF7CCFC0C222900601C07F0D5F80D20D7
:1048600030E0722800D174E0DC2800D1A9E0DB2818
:1048700000D0C3E0042DCED9B278737812021A4367
:10488000F37810271B041343327912061A4301925E
:10489000052D05D06F1F3A000198711D07F0B4F87F
:1048A00005223100200007F0AFF83A000199601DA1
:1048B00007F0AAF8781D05E00C222000674907F0F0
:1048C000A3F80C2005B0F0BD0C22B8E70C22644917
:1048D000604DB5E7013A634D0C2A11D8002A08D083
:1048E000711C280007F090F80C2228005E49FEF7A2
:1048F0007DFC13222900601C07F086F81420E1E7F4
:104900000C22EDE7574D1322280007F0B5F8FEF70B
:1049100077FBEEE705225549601C07F075F8062085
:10492000D0E712225249601C07F06EF81320C9E745
:1049300008225049601C07F067F80920C2E7717827
:10494000F72900D967E74C4B188801F0C1FC022019
:10495000B8E700F09FFB012D02D07278474B1A6038
:1049600006F0F2FE0020ADE7013A454D062A0ED8CA
:10497000002A05D0711C280007F046F800F0C2FF9D
:1049800006222900601C07F03FF807209AE706225C
:10499000F0E7013A3B4D042A11D8002A06D028003E
:1049A000711C06F049FF384B1B68AB60FFF77EFEB9
:1049B00004222900601C07F027F8052082E7042262
:1049C000EDE7022A00D826E773786370B378A37006
:1049D00077781B021F43032A05D0033D3900AAB292
:1049E000F01CFEF703FC10223900E01CFEF7C4FCAB
:1049F00003000330002B00DB64E70DE7DA2800D06A
:104A000009E7042D00D806E7B37872781B02134338
:104A1000F27812041A4333791B061343082D16D972
:104A2000B279717912020A43F17909041143327A99
:104A300012060A4303921A601B6805223100200007
:104A4000039306F0E1FF0422601D03A973E7FE2231
:104A50006270F1E70C63FF1FFC0C0000E0BB00116B
:104A6000D4BB0011E862FF1FF50C0000F462FF1FC9
:104A7000D462FF1F9C44FF1F5E43FF1F34F00040C1
:104A8000F943FF1F1863FF1F28F00040704770476D
:104A9000013870B5042809D806F076FD0309250809
:104AA00012001B4B0221187806F016FE70BD184B41
:104AB0000821187806F0E8FD0022164B1A72F5E777
:104AC0000024144B124D08211A6828781C8106F026
:104AD0006BFF2100287806F0CFFD012000F04CFE8E
:104AE00000F010FFE2E70A4B0821187806F0CCFD31
:104AF0000948FFF7C1F9094B094A9B7900209380C7
:104B0000084A13808022034B52001A81E6E7C04610
:104B10002863FF1F2C63FF1F6743FF1F0C63FF1FEA
:104B20002845FF1F0465FF1F020010B5094B0A321C
:104B3000094C92B2DA815A8298811882207802F068
:104B40002DFA0422054B012120781A7006F0C4FDCD
:104B500010BDC0462644FF1F6665FF1F6565FF1F29
:104B600010B5012909D1054B1B78002B05D0262251
:104B7000034B04485A72FFF7D7FF10BD3865FF1F7B
:104B80002C63FF1FC409000010B5164C0A21022334
:104B9000E05E06F0E9FE00B200F00AFE0423E05EEB
:104BA000642106F0E1FE012100B200F071FE237ADB
:104BB0000024132220009A426041C0B200F0EAFDB6
:104BC000032000F0AFFD200000F0C0FD064B187878
:104BD000053843425841C0B200F0CEFD00F092FECD
:104BE00010BDC0460063FF1F6565FF1F0300F0B5E1
:104BF0000A4D8E18B14202D152008018F0BD0C78D7
:104C00002F6824093C5D0F271C700C7801313C4053
:104C10002F683C5D5C700233ECE7C0465443FF1FD5
:104C200010B5114B1A781870002A0ED000280BD13D
:104C30000E4B1A78062A07D85423D340DB0703D536
:104C40000B4B187802F0AAF910BD0028FCD0074BD6
:104C50001B78012B02D0033B022BF5D8044B01211A
:104C6000187806F039FDEFE73865FF1F6565FF1F0F
:104C70006665FF1FF7B5614D614A624928700820DB
:104C800005F0E0FB0121022005F0DAFA022005F030
:104C9000C3FB0121002005F0D3FA002005F0BCFB86
:104CA00000F05AFEFEF7ACF906F056FE0322564914
:104CB0005648FFF79BFF2D24030004221C70544923
:104CC0000130FFF793FF302302220470437083709A
:104CD000504C514B2000DA8706F096FC022815D084
:104CE000062220004D49FEF747FB06280ED003217F
:104CF000200006F0C9FB8D23E3706E3B2371062272
:104D00001933200045496371FEF770FA0D23444FB3
:104D1000444C454E3B70013B042230004349237014
:104D2000033B6370019606F06FFE2D23012240497C
:104D30004048A371FFF75AFF01223F49FFF756FF92
:104D400001223449FFF752FF0020FFF769FF3B4E75
:104D50003B4A01213B4B1278307802F0E1F8230006
:104D600000213A78307802F0DBF801222178364BC6
:104D700001391A700020019AC9B205F0D7FC334BF3
:104D80001A68552A30D100221A60314B3C32314822
:104D90005A72FFF7C9FE2021287806F0CDFB0120CA
:104DA000404205F00FFD0120404205F0ABFDFFF74A
:104DB00057FAFFF745F800F093FC01204042FFF757
:104DC0000FF9012006F058FDF72001F065FA0121E6
:104DD000287806F081FC287802F03CFA1E4806F09C
:104DE0006BFCFEF73BFFF7BDFA210B4B1B4A490159
:104DF0009981DA8119825A82CDE7C0462863FF1F64
:104E00008D4A0011614B00119C44FF1FD462FF1FAB
:104E1000F462FF1F6509FF1F2644FF1FADAC0000B1
:104E20003465FF1F1565FF1F1765FF1F93BB00113A
:104E30006709FF1F1C65FF1F6609FF1F6665FF1FCF
:104E40008643FF1F6743FF1F0665FF1F34F00040C6
:104E50002C63FF1FC40900003863FF1F4A1F0000B6
:104E6000F8B50A0020230D001A4019423BD0494BE7
:104E70001B78002B23D0FFF719FC474C474E636883
:104E8000727AC31A934202D36060FEF7E7FE327A69
:104E9000217A531EDBB2994214D1FFF779FA637A73
:104EA000002B09D0013BDBB26372002B04D1707977
:104EB00064335843FFF738FE237A013323722020EE
:104EC0006840F8BD9142EAD300232372FFF780FACD
:104ED000FFF75AFE324F3800FEF7CEFF390015209B
:104EE00006F062FCDBE70BB2002B0ADA2D4B1878D8
:104EF00006F0E2FA002801D006F076FB80200002DE
:104F0000DEE70224214206D0234B01201A72FFF76C
:104F100087FE2000D4E70B0715D5FFF7C7FB1E4A15
:104F20001E495368497AC31A8B4202D35060FEF778
:104F300095FEFFF74DFAFFF72BFAFFF725FE00F07D
:104F4000E9FB0820BCE71024214206D0114B1B7856
:104F5000002BDED1FEF788FFDBE7012421420AD0D7
:104F6000114800F06FF806F0A7FC072000F020FCC5
:104F700000F0C8FCCDE74024214202D0FFF7EEF854
:104F8000C7E704240800204021429AD0FFF744F8E4
:104F9000BFE7C0463865FF1F2C63FF1F0C63FF1F70
:104FA0006743FF1F2863FF1F4C43FF1FF0B51B4BD8
:104FB0001B4F1B883A8804001A4E1B4D85B09A423D
:104FC0000DD832889A420AD3184B1A882B889A42F5
:104FD00005D1174A174B12881B889A421BD005200F
:104FE00001F0B0F93B8802AA138033880190538006
:104FF0002B88114D93800F4B02A91B88D3800F4B38
:105000002A78188802F0CCFE0D4B08212878019AE6
:105010001C7006F061FC05B0F0BDC0460265FF1FC4
:105020005C43FF1F5A43FF1F0465FF1F0065FF1FFE
:10503000FE64FF1F5843FF1F6665FF1F5E43FF1F8F
:10504000FC64FF1F13B50C4B1C78002C11D10028F9
:1050500001D00A4B18600A4A0A4B11780A4A1078A4
:105060000A4A01920A4A0092002205F057FA2000EB
:1050700016BD1124FBE7C0466565FF1FF864FF1FDE
:105080006465FF1F5465FF1F6665FF1F4065FF1FB6
:105090004465FF1F10B5064B12201B78052B06D167
:1050A000044B13221988044B187801F027FB10BD1C
:1050B0006565FF1F5E43FF1F6665FF1F10B5002477
:1050C0000122114B52421870104B1C70104B1A8069
:1050D00002F0C0F804220F4B21001A700E480C3267
:1050E00006F0CAFC102221000C4806F0C5FC07227D
:1050F0000B4B1C600B4B1C700B4B1C700B4B1A703A
:105100000B4B1C7010BDC0466665FF1F6565FF1F19
:105110005E43FF1F6465FF1F5465FF1F4465FF1F4B
:105120004065FF1F1465FF1F1365FF1F6043FF1FCE
:105130001265FF1FF8B5174C0600257806A8142441
:105140000078052D23D1B41F134FA5B21824BD42FA
:105150001DD88D1FADB2BD4219D8FA256D00AA42E7
:1051600015D21D000D4F0A3DADB2BD420FD80C4CFB
:1051700026800C4C21800C4900240A800B4A1380A5
:10518000FFF714FF0A4B0421187806F07DFA20007F
:10519000F8BDC0466565FF1F790C0000750C000066
:1051A0005C43FF1F5A43FF1F0465FF1F5843FF1F47
:1051B0006665FF1FF0B50BB20D0089B0002B00DB58
:1051C00076E1A64E307806F077F9041E55D00378C4
:1051D000A22B00D127E1D02B1AD0912B4AD14378B2
:1051E0000E2B47D19E4B82889A4243D19D4A8368B9
:1051F0001278052A3ED1032018567F283AD09A4BC0
:105200001B68002B36D05B68002B33D0984731E009
:10521000807807282ED806F0B7F9042D1D4444796C
:10522000ADDD6378002B11D10622E11C8F4806F01A
:10523000EBFB01218B4B19708D4B1A78002A5BD048
:105240008C4B307801F06CFE002855D00722854B3E
:105250001A7051E061780029F8D1E378002B11D061
:10526000854A864B1278307801F05AFE6070637878
:10527000002BEBD1200006F0B7F980200002684037
:1052800009B0F0BD774B1B78022BF3D001213078A9
:1052900006F082F90028EAD10121307806F01CFAE4
:1052A000E5E76378002BD1D16E4F032807D13B7817
:1052B000052B02D101333B701EE00223FBE7704B4C
:1052C0001A88704B0293002A0BD01B78002B03D056
:1052D0000121307806F000FB3B78062B04D1013B1E
:1052E000E9E7029B1A70F7E7042B41D10121029BE9
:1052F0003078197006F0F0F95B4B1B68002BB9D0C1
:105300001B68002BB6D0574A10787FE76378554F5B
:10531000002B27D10622211D5B4806F075FB628910
:105320005A4B5B491A80A2895A4B1A80E3890B8039
:105330000521397058490A80584A1380228A584BEF
:105340001A80584B1B78012B09D11F2000F0FAFF5F
:10535000FA22920042430421307806F0BDFA00227E
:10536000484B75E7312B00D070E70022454B1A708F
:105370000323A0E706220021434806F07DFB00231B
:10538000454A04211380454A30781380444A1380EB
:1053900006F07AF90821307806F076F9A379083B0F
:1053A0005A4253412F4A03331370314B1B78002B61
:1053B00006D0344B30781A78002A06D001F0EEFD82
:1053C0000122324B52421A8096E70121197006F0F1
:1053D00083F9F5E70821307806F056F96378002B59
:1053E00000D047E72C4B2E4F0293E388029A04210A
:1053F00013802A4B307803932389039A138063899F
:105400003B8006F0C9F8002800D033E7264B1B6824
:10541000002B00D12EE7039902983A88098800886A
:105420001B68984726E74379132B00D022E70389AE
:10543000012B0AD11D4B1B78022B06D10821307895
:1054400006F022F9FFF726FE14E7052000F07AFFA8
:1054500008210200307806F03FFA0BE76665FF1F6F
:10546000051400006565FF1FF864FF1F3965FF1F05
:105470008643FF1F6743FF1F3465FF1F1565FF1F2E
:105480003665FF1F3865FF1F0765FF1F5E43FF1F5F
:105490000E65FF1F1065FF1F0265FF1F0065FF1FE0
:1054A000FE64FF1F0665FF1FF464FF1FFC64FF1FFF
:1054B0008020C001014200D0E1E6CB0731D5324B5C
:1054C0001B78002B1DD0314E05AC3378052B1AD13B
:1054D000023B23702E4B21001B7823722D4B1B782F
:1054E00063722D4B187801F0BFFC002809D007200B
:1054F0002A4B30701B68002B03D01B68002B00D098
:1055000098470120BBE60E20254B06221B78254933
:105510002370254B1B78637002ABC01806F074FA39
:10552000D8E7022308001840194209D0174B1B780E
:10553000052B03D11D4B188806F086F802209EE645
:105540000424214203D0FFF731FD200097E6082311
:1055500008001840194200D192E6154B1C78012C26
:1055600003D0022C0DD0082089E6124B124A1349B1
:1055700013481B881288098800880094FFF7DAFD19
:10558000F1E7FFF787FDEEE73865FF1F6565FF1F51
:105590006043FF1F1265FF1F6665FF1FF864FF1F52
:1055A0001465FF1F6143FF1F1365FF1F5E43FF1F4D
:1055B000FC64FF1F5843FF1F0465FF1F5A43FF1F72
:1055C0005C43FF1F10B502A804880B20002C10D1EB
:1055D000496808784978090201430C48814209D199
:1055E000022119800A4B59881170DB7800205BB2C8
:1055F000537010BD074C0A20A142FAD10221198034
:10560000034B998811705B79F0E7C0466E2A000061
:105610000063FF1F6F2A0000F7B5150008AA16885F
:105620004A680F4F14785278120222430A24BA4271
:1056300014D10122DBB2019200962A0005F074FE1B
:10564000041E0BD1074B1B68002B07D068782A7803
:105650000002104342425041013098472000FEBDF5
:10566000022900007865FF1F30B501250379040089
:10567000BFB02B4227D01549408805F0C1F9284218
:105680000DD06A46124B69465B8D1380022353800E
:10569000104B5B8893806088002202F077FA0E49F5
:1056A000608805F0ADF9C0070DD56A460B4B694619
:1056B0001B88138002235380064B9B88938060884D
:1056C000002202F063FA3FB030BDC0467065FF1F94
:1056D0008843FF1F0063FF1F6865FF1FE243FF1F32
:1056E00010B5074C0749200005F040F92000064995
:1056F00005F03CF90721054A054805F0F9F810BD09
:10570000FFFF00007065FF1F6865FF1F60BC001190
:105710008843FF1F10B5024803F0BAF810BDC04619
:105720006956001170B55F25082607498400CA78BC
:105730008B7840012A40B3433440A84323430243BB
:105740008B70CA7070BDC046F943FF1F010043B2A1
:1057500004205A0002409B000C3003401A431523DA
:1057600010B5044CE0789843143B0B4018430243B7
:10577000E27010BDF943FF1F10B5054B08241979DD
:105780000A00A243002801D022000A431A7110BD6A
:10579000F943FF1F10B5054B4024D9780A00A243F6
:1057A000002801D022000A43DA7010BDF943FF1F20
:1057B000082170B5314D0400AB780B40AB70304B15
:1057C000984204DD67232B70473B6B7070BD2D4BF7
:1057D000984203DAE0232B703A3BF6E700232B7064
:1057E0006B7083B21A0028485F3292B2274E824211
:1057F0002CD9002C03DA5B421CB204232B70053435
:1058000020B20A2106F0B0F804B2FA239B009C42B1
:1058100031DB08232A7813432B706421200006F023
:10582000A3F80A2100B205F01FFE09B22A78735CC2
:1058300013432B700A21200006F096F80A2100B2CB
:1058400005F012FE09B2735C6A780AE06970002CF8
:10585000DBDA5B421CB204232B70F3226B78092C39
:10586000E8DC13436B700A21200005F0FDFD09B24E
:10587000735CAB70AAE7632CCFDCEEE7F943FF1F44
:105880001B4E00001DFCFFFF2A08000087BC001112
:105890000823F7B5194FCD003E7904001E403E7134
:1058A000EDB2632806DD183333433B7167231D4394
:1058B0007D71F7BD0300093305DA5A235B42334398
:1058C0003B71E023F3E70E4B019300280BDA04232E
:1058D000444224B23B710A21200005F0C5FD019B22
:1058E00009B25B5CE3E70928F5DD0A2106F03CF824
:1058F000019B00B21B5C1E433E71ECE7F943FF1FA6
:1059000087BC001170B5104B1B78002B1AD00F4EBE
:105910000F4D06223100280005F016FE002811D098
:10592000062231000B4C280005F086FF0020FEF710
:1059300063FD072221003E20FEF78CFE002801D0E7
:10594000FEF7CEFD70BDC0468365FF1FF943FF1F04
:105950007D65FF1F7C65FF1F002010B5FEF74CFD25
:105960000D223E200549FEF775FE0023984200D126
:105970003E33034A1370FEF7B3FD10BD7ABC00112D
:105980008365FF1F0200F0B501270A480A4E51182F
:105990008B1A002B00DCF0BD082415784308684002
:1059A00038404000805B013C58406D08002CF5D128
:1059B0000132EDE7FFFF000098BC0011F0B50025B3
:1059C0000F269D4200DBF0BD4C5D0709444034408A
:1059D000A400A05801357840F3E70000F0B589B085
:1059E0006A460D000B000F27110010351C7801339B
:1059F000260024093E40167054700232AB42F5D1A5
:105A00002023024AFFF7DAFF09B0F0BD9CBC001169
:105A1000F0B54E780B7889B036020C001700019073
:105A20001E43012A61D9974B9E4200D877E001338B
:105A30009E421CD1062A17D1CA788B7812021A43CB
:105A40000B791B0413434A7912061A438E4B5A6191
:105A500000221A705A808D4A5A608D4A9A608D4A87
:105A6000DA60002009B0F0BD88225205EEE78A4BCB
:105A70009E423CD184498B78002B00D0F9E00C2A5F
:105A800031D10F22A3789343E27812021343227993
:105A9000120413436279120613434B60E279A07932
:105AA00012020243207A00041043627A1206024373
:105AB000CA60E27AA07A1202024378484A8183429D
:105AC00008D804237049142201980B7005F09CFF3C
:105AD0001420C7E71201D21889235B059A42F0D837
:105AE00001238B70BDE7022AFAD00523EAE76C4A4E
:105AF00001239642E6D1FFF7CDFA052F0CD9E378C2
:105B0000A2781B021343227912041A4363791B06FD
:105B10001343644A0393136005F016FEA1E75A4D40
:105B20002B78002B9DD1AB78002B00D1A3E02B89E3
:105B300001339BB20093B34200D094E0132AD4D92E
:105B4000CF7C8B7C3F02122120001F43FFF71AFFFE
:105B5000874200D091E0002E3ED1E378A2781B026C
:105B600013432279E96812041A4363791B0613432D
:105B700003930A228B4213D1FF23A370E370237196
:105B800063716B89002B0AD1E37B227C1B02120418
:105B90001343A27B134303931B0901336B81002240
:105BA0006B89002B8DD0002A69D1686837013818BD
:105BB000000B6B6900030390984205D9686105F0FA
:105BC000B3FDEB780133EB7068681022A11C381824
:105BD00005F042FF2E8144E76F89009A7B1E9BB23D
:105BE00093423CD1E378A2781B02134322792E4ED4
:105BF00012041A4363796C681B06134331000422B4
:105C000004A8039305F000FF211D0C2205A805F050
:105C1000FBFE012004A940421034FFF7DFFE013FE4
:105C2000012F17D1039A0B232861824200D049E744
:105C300004223100686805F00FFF042203A9686898
:105C400005F022FFE968039AFF23914200D139E76A
:105C5000F73B37E72100FFF7C1FE1034DFE70923E8
:105C6000B742A2D82EE7009BB34200D9F9E607233A
:105C700028E7022326E7032324E7062322E70A2353
:105C800020E7C046FFFE00000044FF1F0000011196
:105C9000FFFF00005048593601FF0000FFFF0011D0
:105CA00002FF000034F000400C44FF1F10B5034C0D
:105CB0000B000122210000F06BFA10BD6D5E001197
:105CC0000B8870B506000D000224162B11D92B008D
:105CD0000322094900F05CFA041E0AD1074B2A8806
:105CE0001B88191C934200D9111C300089B200F0A6
:105CF000EFFA200070BDC046995E0011DE65FF1FFF
:105D000010B54A780400013A0B000220012A07D896
:105D10000A78002A04D005222000024900F038FA4F
:105D200010BDC046C75E00110A7810B50B00040014
:105D30000220002A04D007222000024900F028FA9D
:105D400010BDC046735F00110A7810B50B00040047
:105D50000220002A04D009222000024900F018FA8B
:105D600010BDC046D95F001110B5034C0B000B22CB
:105D7000210000F00DFA10BD0960001110B5034CB0
:105D80000B000D22210000F003FA10BD7B60001112
:105D900010B5034C0B000F22210000F0F9F910BDE3
:105DA000D56000110A7810B50B0004000220002A0B
:105DB00004D011222000024900F0EAF910BDC046CB
:105DC000E5600011002310B51322190000F0E0F97E
:105DD00010BD000010B5034C0B001722210000F08D
:105DE000D7F910BD37610011002310B51922190031
:105DF00000F0CEF910BD000010B5034C0B001B22C3
:105E0000210000F0C5F910BD71610011F7B584895A
:105E10000D0006000121002C22D000238268D356F9
:105E20001778002B1EDA0C2C1AD90C3CA4B21319CB
:105E300040880093230002F086FE431E9841013003
:105E40007B06DB0F6B703F23013C1F40A4B2287020
:105E5000AF70AC80002C07D0B3680133AB60002179
:105E60000800FEBD0020EBE7AC60F8E70B7803709C
:105E70004B8843704B881B0A83700B79C3700420D6
:105E800070470420022B06D10020537811781B02A2
:105E9000009A0B43138070470B8803700B881B0A12
:105EA0004370022070470420009983420AD153783E
:105EB00010781B0203430B80D37890781B020343B6
:105EC00000204B807047F8B50D004B78012400216D
:105ED000461C03702B788B4201D82000F8BD6B78EC
:105EE000B01C4F1C012B10D1890069184B8802226D
:105EF00033704B88B9001B0A7370691805F084FD74
:105F000004360434A4B2F9B2E4E7122359436B18FF
:105F10005A88043132705B8810221B0A737069182A
:105F200005F072FD12361234ECE770B5049D1400D2
:105F30001E00052B01D8042070BD637812781B0267
:105F400013432B80E378A2781B02134302226B8059
:105F50002A71211D681D063E05F056FDB2B22A8148
:105F6000F02AE8D82800A11D0A3005F04DFD0020D8
:105F7000E2E7002310B50A789A4201D8900010BDDC
:105F80009A008A185488013304705488DBB2240ABA
:105F90004470948884709288120AC2700430EAE7D0
:105FA00010B51100029C062B04D004201022142BE3
:105FB00001D010BD022222714B7808781B020343E6
:105FC0002380CB7888781B02034363800431601DF3
:105FD00005F01AFD0020ECE710B50C788B78043141
:105FE0005C43E4B203702200013005F00DFD601C3B
:105FF00010BD0420022B06D10020537811781B021B
:10600000009A0B431380704710B50C000A880231C8
:1060100005F0FAFC208810BD70B504000D0004984E
:106020001100012B01D8042070BD1678527812029D
:10603000324302800200F83255701470E825002CBB
:1060400000D10C35023B9AB24280AA42EBD8023111
:10605000043005F0D9FC0020E6E7042000998342D3
:106060000AD1537810781B0203430B80D3789078C1
:106070001B02034300204B80704710B50C000A88B8
:10608000023105F0C1FC208810BD000070B501216F
:106090001E000420049C0E400B4218D1CB40DDB200
:1060A0008D4214D90A49DBB2098899420FD32300E3
:1060B000F6331D703300580011184978165C090238
:1060C000314301332152D9B28D42F4D8002070BD42
:1060D0002044FF1F10B50C000A88023105F094FC23
:1060E000208810BD10B50C788B7804315C43E4B285
:1060F00003702200013005F087FC601C10BD10B554
:1061000011000298032B01D8042010BD1478527896
:10611000043B120222430280CA788C781202224386
:1061200042809AB28280F22AEED80431063005F01D
:106130006BFC0020E9E710B50C000B8803700B889E
:106140001B0A43704B8883704B881B0AC3708A8874
:106150000430063105F058FCA088043080B210BD30
:106160000420012B03D100201378009A137070478C
:1061700010B50C000B8803700B881B0A43704A880B
:106180000230043105F040FC6088023080B210BD5E
:10619000F0B589B003931E4B029242000700D05A1B
:1061A000019102F020F81325061E2DD0029B012438
:1061B0000370019B002B04D0001903999847001924
:1061C00084B26B461B7A5BB2002B0FDA10213800C9
:1061D00002F01CFB1925002813D130003219E1B25E
:1061E00002F066FC051E0CD10C34A4B2042304AAF0
:1061F000380005A993800696948101F0AFFD051E35
:1062000002D0300005F020FC280009B0F0BDC046E7
:10621000DC65FF1F70B505000C0000280CD00020C5
:10622000814209D010222000044905F0EDFB012035
:106230002B7823736B78637370BDC046DCBC001190
:10624000F0B506000D0017001C0085B002291BD018
:106250000020102907D1022B07D0102B03D115E005
:106260000020102C08D005B0F0BD69463800FFF7BB
:10627000D1FF2A0069460BE069463000FFF7CAFFEC
:1062800022006946380004E0022BE9D12A003900D7
:10629000300005F031F9E6E7031CF72800D9F723B1
:1062A000032008499AB2013A0B80D31703400649EC
:1062B0009B189B100B80D30F04499B185B100B801D
:1062C0007047C0462444FF1F2244FF1F2044FF1F85
:1062D000034B1B888B4202D3024B4000C1527047D4
:1062E0002444FF1FDC65FF1F014B4000185A704714
:1062F000DC65FF1F1722014B1A807047DC65FF1F0A
:1063000070B505000E2005F0D7FB041E13D0D02376
:10631000037000230622837007494570033005F09F
:1063200073FB064B2100DA8A62811B7E2373044BC8
:10633000187805F049FB70BDF865FF1FE865FF1F81
:106340007444FF1F262803D8024B4000C05A7047F0
:106350000148FCE72644FF1FFFFF000070B5060060
:106360000C00094D1C220021280005F085FB074B7D
:106370001E70074B1C7005F0B7F90123002801D0EF
:10638000002312202B7070BDE865FF1F7444FF1FAF
:106390000966FF1F70B505000D4C0800E260A160A2
:1063A00010220021656005F047FB012803D1102170
:1063B000A06802F058FD10220021280005F03CFBE7
:1063C000012803D11021606802F04DFD70BDC04668
:1063D000E865FF1F70B5041E05D1002903D0062211
:1063E0000D4805F011FB0D4B1D78012D11D1002C2E
:1063F00005D102221A7005F0BFF9280070BD0022F5
:106400001A70074B1B78FF2BF7D02000FFF778FF9F
:10641000F3E70025F1E7C046F865FF1FE865FF1FB9
:106420007444FF1F030010B5002801D1002010BDE7
:1064300000780B4A002803D15988D1821B79137642
:106440001378022BF2D10023984200D1033313704A
:10645000044B1B78FF2B01D0FFF752FF0120E6E72A
:10646000E865FF1F7444FF1F002911D000280CD0DD
:106470004B79012803D140225242134303E03F22CB
:106480001340032802D001204B7170474022F4E7EB
:106490000800FAE770B5094D0100287800280BD0F4
:1064A000074C0622200005F0AFFA21002878FFF7FC
:1064B000DBFF200005F0B0F870BDC0460866FF1F86
:1064C000E265FF1F00290AD0012808D13F224B793D
:1064D0009343C02B03D0403B5A425341981C704712
:1064E00070B5174D06002B78FF2B15D00A2005F04C
:1064F000E3FA041E10D0D0230370C83B8370114B05
:1065000011491B784670C3700622043005F07CFAEE
:106510002100287805F058FA0C4B1B78012B0DD17F
:106520000B4B1B68002B03D09B68002B00D09847B7
:10653000084B04211878084A05F036FA70BDC046A9
:106540007444FF1F0866FF1FE265FF1F0466FF1FFC
:106550003066FF1F3466FF1F60EA0000014B986839
:106560007047C046E865FF1F014BDB68186870473D
:10657000E865FF1F074B10B5DA6813680133136035
:10658000054B1878FF2803D08021C90105F0A4F835
:1065900010BDC046E865FF1F7444FF1FF7B50E002D
:1065A00002F0C8F8051E1CD00E4B06621F78002FA3
:1065B00000D10778AB791020019305F07DFA041E15
:1065C0000FD0D0230380C73B8370019BE91DC370AC
:1065D0000622043005F018FA21003800E66005F0C4
:1065E000F3F9F7BD7244FF1F014B18787047C0469E
:1065F0000866FF1F054B002805D1054B1A78054B8F
:10660000002A00D1014B18007047C046F865FF1FF3
:106610000866FF1FE265FF1F014B58687047C046C0
:10662000E865FF1F024B1868431E9841C0B27047CF
:106630000C66FF1F421E03000120152A03D9FF3BF1
:106640005A425341D8B27047F0B51C0000230E00E7
:1066500085B0039002920B70029A934201D30020FE
:1066600019E0E55C5A1CD2B2002DF8D002985119FD
:106670008142F4DC0233DFB2A35C18000193FFF720
:10668000D9FF002807D0013D019A0399EBB233707E
:106690008A4202D1E01905B0F0BDDB19DBB2DBE7BD
:1066A00010B50C0002F09EF803001220002B03D05E
:1066B0002100588804F0E0FE10BD000070B50E4DBA
:1066C00084006359002B15D0186A002801D004F00B
:1066D00093FF2B59586A002801D004F08DFF2B59E5
:1066E000986A002801D004F087FF285904F084FF3D
:1066F00000232B5170BDC0461866FF1F1C4B70B5A0
:1067000004000E00150099420AD11A4B1B68002B99
:1067100001D1122070BD1B68002BFAD09847F9E711
:10672000154B994215D1134B1B68002B0AD01B68DF
:10673000002B07D09847002804D1104B1C70104B39
:106740001D70E7E729002000FFF7AAFF0028E1D12C
:10675000F3E7080001F0EEFF0028DAD00378032009
:10676000A342D7D12900300004F086FED2E7C0460C
:10677000FEFF00001466FF1FFFFF00001166FF1FF1
:106780001066FF1FF7B50400808801F0D3FF0025D5
:10679000A84203D00578A08802F008F81C4E337890
:1067A000002B1FD0AB421DD11A4B28001978FFF7E0
:1067B00077FF002818D000233370A3790820A7782A
:1067C000A688019305F078F9011E0DD0D02303703F
:1067D000CA3B8370019B477086808371280005F057
:1067E000F3F801E0002DE8D1A0880B4B8200D358CC
:1067F000002B01D0FFF762FF1721A088FFF768FD8B
:10680000A08801F027FDA08801F0FEFDF7BDC0467D
:106810001166FF1F1066FF1F1866FF1FF0B587B0D7
:106820001D000CAB1B88070001930DAB1B881420C7
:1068300002930EAB1B88160003930FAB1B880091CD
:10684000049310AB1B88059305F036F9041E1AD08B
:10685000D0230370CB3B47708370C670062229009B
:106860000430002D11D005F0CFF8019B2100638189
:10687000029B0098A381039BE381049B2382059BD9
:10688000A37405F0A1F807B0F0BD05F0F5F8ECE74A
:10689000F7B5009308AB1B8807000C200D0016000D
:1068A000019305F009F9041E13D0280001F042FFFE
:1068B00000280FD00078D0232370C93BA370009B21
:1068C00021002381019B6770A580E680638105F02C
:1068D0007BF8F7BD014B1878EDE7C0467444FF1F05
:1068E00013B5040064890389C2888188C078009444
:1068F000FFF7CEFF13BD000010B5044C2068002840
:1069000003D004F079FE0023236010BD1C66FF1F36
:10691000A122F0B5818892004A43384B384F1B685A
:1069200004009B189D2292009B18827989B01A60FE
:106930003B68002B5FD01D78324B1B68002B04D0C6
:106940005B68002B01D000209847260008363100F4
:10695000E079FFF7B7FD237DE0710200E078049352
:10696000638A29000393238A0293E3890193A3880E
:1069700000933300FFF752FFE378002B0BD1E2893D
:10698000A379A18802920196E2792800009201225F
:1069900001F0DAFEE0703B68002B20D0FFF7ACFF7F
:1069A000194D287800281AD0184B1978FFF778FE6F
:1069B000002814D02B78E67808200793A78805F0E4
:1069C0007BF8011E09D0D0230370CA3B4670837048
:1069D00087808671079804F0F7FF00232B7017213A
:1069E000A088FFF775FCA08801F034FCA08801F0B6
:1069F0000BFD09B0F0BD064B9DE7C0463409FF1FF3
:106A00001C66FF1F3066FF1F1166FF1F1066FF1F09
:106A10007444FF1FF8B5070008000E0001F08AFE5D
:106A2000041E18D02620FFF78DFC051E00D1257806
:106A3000062005F041F8041E0DD00021062205F0C5
:106A40001BF8D0232370C23B21006770A370A6807F
:106A5000E8B204F0B9FFF8BDF0B585B001930AAB18
:106A60001B78070002930BAB1B7808000D00009207
:106A7000039301F05FFE061E22D0102005F01CF8E3
:106A8000041E1DD01022002104F0F6FF2620FFF77F
:106A900059FC002800D13078D0232370C13BA3706B
:106AA000009B21002372019B67706372029BA5808B
:106AB000A372039BC0B2E3720C9BE36004F084FFFB
:106AC00005B0F0BDF7B50D00019001F033FE071ED3
:106AD00020D00E2004F0F0FF041E1BD02620FFF76C
:106AE00031FC061E00D13E78D0232380C53B062210
:106AF000A370F91DE01C04F087FF019B2A0063814D
:106B00000123DD401A401D40210022736573F0B25D
:106B100004F05AFFF7BD0000F0B585B002901000F8
:106B20000D0017000A9E039301F004FE041E31D0ED
:106B3000029B002B2ED1039B02795B0724D51223E5
:106B400013430422002E08D10B99002905D10C997A
:106B5000002902D10D9900291AD01A430D9B2271E8
:106B6000002B00D0C9E0002E00D1CFE0002D00D0D6
:106B7000CCE0606A002801D004F03EFD1C2130000A
:106B800004F06AFC606205E002239A430E33D7E703
:106B900093432371654BBA00D458002C00D1AAE06E
:106BA000002E10D0236A002B03D11C2004F004FF18
:106BB00020625E4BBA00D358186A002803D01C220A
:106BC000310004F021FF0C9B002B12D0574CBB006E
:106BD0001D596B6A002B03D1162004F0EDFE68628C
:106BE000BB00E358586A002803D016220C9904F021
:106BF0000BFF0D9B002B11D04C4DBC006659B36AA6
:106C0000002B03D1142004F0D7FEB0622B59986AF0
:106C1000002803D014220D9904F0F6FE380001F08C
:106C200089FD051E67D0414BBA00D358002B62D0B6
:106C30001A6A3420002A00D11C389A6A002A01D02E
:106C4000143080B20B9A002A01D01C3080B25B6AEB
:106C5000002B01D0163080B204F02EFF041E4AD063
:106C60001822002104F008FF2620FFF76BFB01909B
:106C7000002801D12B780193D0232370029B2000A0
:106C800063700A23294EA370039BBD00A371AB5907
:106C9000A780196A1830002905D01C22A06004F0D2
:106CA000B3FE200034307359996A002907D00300DD
:106CB00014221433E060029304F0A6FE02980B9BAA
:106CC000002B08D003001C221C330B992061029377
:106CD00004F09AFE02987359596A002903D01622CB
:106CE000606104F091FE6B462100187904F06CFE9F
:106CF0003800FFF7E3FC05B0F0BD10220D9B0D99A5
:106D00001B69A018236204F07FFE2CE70B9B002B6D
:106D100000D13FE7012D00D03CE7606A002801D098
:106D200004F06AFC1C210B982AE7C0461866FF1F76
:106D300010B5044C2068002803D004F05DFC00234B
:106D4000236010BD0C66FF1F0B4B07B51A68002AA5
:106D500001D100200EBD6946531C01201278073175
:106D6000FFF772FC0028F4D00278012310001840CD
:106D70001A42EED0EEE7C0462866FF1FF0B51F4F5F
:106D800001203B6887B0002B25D09B78059300F04D
:106D9000B3FB002821D00A20FFF7D4FA04000B200F
:106DA000FFF7D0FA164B05001E78731E9E413B6814
:106DB000F6B2191DD878FFF757FB3B682900DA7A3D
:106DC000043303929A7901930292009033002000D9
:106DD000059A04F0E9FB07B0F0BDFFF7B5FF002806
:106DE00005D00620FFF7AEFA04000720D8E70820F8
:106DF000FFF7A8FA04000920D2E7C0460C66FF1F7F
:106E00000866FF1F70B50A4E040033780D00FF2B93
:106E10000DD0042004F050FE011E08D0D0230370D2
:106E2000CE3B45708370C470307804F0CDFD70BDEA
:106E30008444FF1F70B5040006200D0004F03CFEE2
:106E4000011E0AD0D0230370CD3B8370054B4470E4
:106E50001B688580187804F0B7FD002C01D0FFF77F
:106E600067FF70BD0C66FF1FF8B5264F06003B6834
:106E70000D001124002B05D10522234B1B78134252
:106E800002D112242000F8BD204A10241268002AE2
:106E9000F8D01278002AF5D0DB0719D52B789A1E86
:106EA000012A1AD80C2004F087FD1324386000282A
:106EB000E8D000230A22437029000670023004F053
:106EC000A3FDFFF75BFF041E0AD0FFF731FFD9E7F0
:106ED00000F012FB0028E1D1E4E7002BE2D0D0E77C
:106EE0000B4B1B78032BCDD11D20FFF72BFA094B41
:106EF00018800028C6D0084B04211878074A04F0EF
:106F000053FDBFE70C66FF1F0966FF1F2866FF1FC2
:106F10000866FF1F0666FF1F3466FF1F60EA000059
:106F2000F7B50193194B14001A78052306000F00DA
:106F300012201A4221D0012920D1154B1D68002DA5
:106F40001BD002201F2C18D8002C02D0019B002B34
:106F500013D0104B1F221E706E1C0021300004F055
:106F60008BFD01992200300004F04EFD310020001D
:106F70002C70002F06D004F0BFFBFEBD064B122084
:106F80001D68DCE704F0D8FCF7E7C0460966FF1F80
:106F90002866FF1F8444FF1F2466FF1FF8B50F4EAD
:106FA00012243368002B17D01B780F3C834213D177
:106FB00000250B4F0221387804F066FB094B0421B1
:106FC00038781D8004F060FB074B28001D80336873
:106FD0005C7004F061FB04002000F8BD0C66FF1F2C
:106FE0003466FF1F2066FF1F0666FF1F70B501286D
:106FF00023D11B4C2388002B03D01A4A1578002D6F
:1070000007D0194B1B68002B02D01878FFF7C6FF7A
:1070100070BD3B2B02D93C3B2380F9E7134E022184
:10702000307804F031FBFA222388920002215A437F
:10703000307804F051FC2580EAE70B4B1B68002BED
:10704000E6D00B4B1B785B07E2D5084B0221187882
:1070500004F01AFB0022024B1A80FFF769FED7E703
:107060002066FF1F0466FF1F0C66FF1F3466FF1FAC
:107070000966FF1FF8B51E4D2868002803D004F0EC
:10708000BBFA00232B601B4E3068002803D004F0AD
:10709000B3FA00233360184F05243B7818002040D2
:1070A000234221D0154800F02BFA3B78234213D01D
:1070B000202004F081FC2860002813D02022002129
:1070C00004F0DAFC202004F077FC041E306005D0C8
:1070D0002022002104F0D0FC002004E0286804F005
:1070E0008BFA2C601320F8BD00F00AFAF4E7C046D2
:1070F0002866FF1F2466FF1F0966FF1F7844FF1FD5
:1071000010B50A4C23681A1E0ED0002808D1013091
:10711000587004F0C1FA002805D02368002B02D073
:107120000021FFF787FE0122100010BD0C66FF1F33
:10713000F7B5274E050033680191181E21D05C7801
:10714000244F012C30D1FFF7FFFD002825D020006F
:10715000FFF7F8F80400412814D91F4B02211878D2
:107160001E4A04F021FC1E4B3C3C1C80022233686A
:107170005A703B78002B14D128000199FFF75AFE72
:107180000120FEBDFA2292004243002AEED0124BAB
:107190000221187804F0A0FBE8E7FFF7D3F802001B
:1071A000F3E700233B70EBE73B78002BE8D10320AB
:1071B00004F082FC011E08D0D0230370CC3B457044
:1071C00083703368187804F0FFFBFFF7B1FDD7E751
:1071D0000C66FF1F0466FF1F3466FF1F60EA000095
:1071E0002066FF1F10B51749838802008B4220D00C
:1071F00011D815498B4217D0144900205B1899B259
:10720000012907D8926811785A425341D8B2FFF742
:10721000F9FD012010BD0E4A00209B1807229BB2E9
:107220009A424041C0B2F5E783681878FFF768FFDB
:10723000F0E7836899785A78090218781143FFF7C4
:1072400077FFE7E70A20000006200000F8DFFFFFD5
:10725000AFDFFFFF014B18707047C0468544FF1F2A
:1072600010B5064C207001F041FA207804F07CFA49
:107270000521207800F062FD10BDC0463466FF1F76
:107280000BB273B50D00002B00DBC4E0884B1878FF
:1072900004F012F9041E0ED00378912B0FD0A22B0C
:1072A00000D1A1E0834B1878FF2852D0210004F0D0
:1072B0008BFB00284DD180200002684076BD4378CA
:1072C0000F2B76D013D8052B70D00E2BEAD18088E7
:1072D000794B98422BD8794B98421BD8784B9842DF
:1072E000E0D1A3681878591CFFF774F838E03E2BFA
:1072F000D8D18378032B74D06CD8012B6ED0022B9D
:10730000D0D1704B1B68002B23D05B68002B20D0A2
:1073100098471EE06C4BC0180C28C3D804F074FAD0
:107320001DC2C2150BC20B0B0B3223C23C00674BB4
:10733000C0180728B6D8664B1B68002B09D01B68FD
:10734000002B06D0200098470AE0A3681878FFF7C2
:10735000C7F8200004F048F9ADE7A068FFF762F82D
:1073600000289FD0F5E7A3681B78002BF1D0554B80
:107370001B68002BEDD01B68002BEAD0210055487C
:107380009847EDE74F4B1B68002BE2D01B68002BA2
:10739000DFD021005048F3E7504B1B68002BD8D0BA
:1073A0005B68002BD5D021004348E9E7FFF7EAF9F5
:1073B000CFE780884A4B984203D04A4B984200D08E
:1073C00070E7464B1B68002BC3D05B68002BC0D016
:1073D0002100D5E7153B012BBBD963E7FFF798FAEE
:1073E000B7E7FFF77DFAB4E73F4B1B78042B07D1D3
:1073F00000236A4613800179408800F0C5FCA8E7A5
:10740000364B1B68002BA4D05B68002BA1D0010079
:10741000364898479DE7012421420AD0294B1B6832
:10742000002B04D05B68002B01D00020984701207E
:1074300043E78B070AD5264B1B68002B04D05B68FB
:10744000002B01D020009847022036E704212800B5
:1074500008400D4200D131E7254E3388002B21D062
:10746000013B9BB23380002B1AD1FFF7DBF80028D9
:107470000AD0204B1C70164B1B68002B04D05B6895
:10748000002B01D020009847FFF7C6F8694601F0AD
:1074900001FD6846FEF7FEFF1D20FEF753FF30801A
:1074A00004200AE7024B187804F0EEF8F8E7C0462B
:1074B0003466FF1F8544FF1F0E20000001200000DE
:1074C000091000002C66FF1FFEDFFFFFAFDFFFFF8C
:1074D0003066FF1F0C2000000B2000001466FF1F09
:1074E0000D200000132000000966FF1FFFFF0000B1
:1074F0000666FF1F0466FF1F10B501F09BF910BD63
:10750000014B18607047C0463066FF1F0B88002093
:10751000162B01D817230420014A13807047C04658
:10752000DE65FF1F00207047074A03001188814273
:1075300007D091880020994202D1013080001018B4
:1075400070470020FAE7C0463C66FF1FF0B58F7811
:1075500006000D00C7B01E2F15D1FFF7E5FF051E71
:1075600003D10024200047B0F0BD00223B003100D1
:10757000C078009200F0B2FB0400A81C00F0D3FB1E
:10758000FF23EB70EEE7264B062403931B78FF2BBB
:10759000E8D0182FE6D87B08224A013BDB00029294
:1075A0009A589446002ADDD0029AD3185B68002BC3
:1075B000D8D00878002802D14B78012B02D10624BC
:1075C000122FCFD107AFAB88697800976446AA68BD
:1075D000A047041EC6D1AB78029A5B08013BDB00D2
:1075E000D318390030005B689847041E0BD1AB7884
:1075F000042BB6D0039A310010782200009700F0D7
:107600006DFB0400AEE76A78002AABD1AA7805A921
:107610003B88087130000A704B80FEF747FBA0E7FB
:107620008844FF1FECBC00111D4B37B50500984284
:107630000BD000290AD1FFF777FF002805D11948A0
:10764000FFF772FF002800D0058037BD01291AD14D
:10765000FFF76AFF041EF8D001235B420380A37882
:10766000FF2BF2D0FE2B07D00023E07814220093EA
:1076700029001E3300F032FBA01C00F054FB012354
:107680005B426380E1E70229DFD1013901F0BEF8F6
:107690000028DAD12800FFF747FF041EDFD1D4E726
:1076A000FEFF0000FFFF0000022210B5074B524210
:1076B0001A80074801325A809A80DA8000F07EFAF8
:1076C000044801F025F8002010BDC0463C66FF1FAD
:1076D0004D750011297600110388F7B50400002BC1
:1076E00002D102252800FEBD4268022113782548F8
:1076F0005268FEF7A5FD00282ED0234F01253A88B9
:10770000002AEFD0802321885B0201259B1A994231
:10771000E8DC0C2004F050F9061E31D03B882288AA
:107720009C4600231800019561469DB2491989B213
:10773000AA421BD8002801D062443A8000233000BE
:10774000082208C0210004F05FF9104A1368002BDA
:1077500013D100251660C5E76268022113780C4832
:107760005268FEF76DFD0028C7D1BAE760681D01B9
:107770004019418101330198D6E71A001B68E6E7FA
:107780001325AFE75ABD00118644FF1F3866FF1F5F
:1077900058BD0011014B18707047C0468844FF1F48
:1077A00014230A0010B51A40194204D001221021F6
:1077B00001F048F810BD4B06F9D401208843400081
:1077C000F8E710B514008B0604D50122102101F052
:1077D00039F810BD08230A001A40194202D14BB2F1
:1077E000002B0FDA102101F02DF8002808D023001B
:1077F000F9331B78002BECD0F8342378012BE8D137
:107800000020E6E703208907FAD4E2E7F0B51F007D
:10781000184B85B01C68019002910392002C27D16F
:10782000200005B0F0BDA5683301ED186B89019A01
:10783000934211D3029A93420ED8002F04D10A9B8F
:10784000002B10D12C00EBE73B002978039A6868E5
:10785000FEF7F6FC0028F2D10136B6B2A388B34297
:10786000E1D82468DAE7A3680A9A5B891380E9E71C
:107870000026F3E73866FF1F37B50C000A884988F1
:107880000123914217D3002A15D0651D23792A00C0
:1078900002210A48FEF7D4FC102300280BD02379DC
:1078A0006188208800242A000094FFF7AFFF0A2394
:1078B000A04200D0230018003EBDC0465ABD0011B2
:1078C00013B50A0008884988012388420BD800288C
:1078D00009D00024137905320094FFF797FF0A239B
:1078E000A04200D02300180016BD13B50A00088876
:1078F0004988012388420BD8002809D00024137935
:1079000005320094FFF782FF0A23A04200D0230033
:10791000180016BDF0B58BB003904A8808880E0099
:107920000123824255D3002853D00023012704AC01
:1079300023700022718813000092FFF767FF051E75
:107940003ED02078002835D12B78022B18D16770D3
:107950006A8983000130E31880005A806968022236
:10796000201804F051F823780133DBB22370042B84
:1079700019D93B006889013080B2002BD9D01FE0B3
:1079800002236370122358436A89231804305A80F3
:1079900069681022201804F037F823780133DBB22D
:1079A0002370002BE5D10C4A6B899B185A42534136
:1079B000DBB2DFE76378012BE4D12B78022BC7D051
:1079C00022780A23002A04D021000398FEF798F9B0
:1079D000002318000BB0F0BD0100FFFF0F4BF0B506
:1079E00004001868002816D083685D89A54207D86E
:1079F0008288AE18B44203DA12019A18934201D178
:107A00000068EFE71E005F891036A74204D1002905
:107A100000D00D801800F0BD3300EFE73866FF1F7F
:107A200070B505000C0008880021FFF7D7FF0300A0
:107A30000120002B04D022002800197AFFF7C1FE94
:107A400070BDF7B50C00002501902300F6331B78BC
:107A5000AB4201D800200AE06B00E65A002130005A
:107A6000E718FFF7BBFF002802D126800130FEBDDA
:107A7000017A0198FFF794FE002802D03B8823800A
:107A8000F5E70135EDB2E0E710B504000888002104
:107A9000FFF7A4FF03000120002B03D02000197A78
:107AA000FFF77EFE10BD0000054B1B68002B01D1C7
:107AB000180004E09A6852898242F6D1988870478B
:107AC0003866FF1FF0B50E27002687B0039302AB80
:107AD000FF183E8005001F4B40891400984207D0D4
:107AE0002B78013000976A6880B2FFF78FFE06009E
:107AF00002212B7818486A68FEF7A2FB00280FD0F5
:107B00006C892000FFF7D0FF002802D0013C041947
:107B1000A4B2039B002B00D01C80300007B0F0BD46
:107B200002212B780D486A68FEF78AFB0028E7D10E
:107B300002212B780A486A68FEF782FB002807D0EA
:107B4000002EDED03B88A342DBD17489013CDFE705
:107B50006C89DEE7FFFF00005ABD001158BD00111F
:107B600056BD001110B50C00FFF7DEFC030002202B
:107B7000002B0AD0002C00D023609B781720FE2B0E
:107B800003D00138FF2B00D1002010BD73B50D00CC
:107B900001A904001600FFF7E5FF172805D0002E05
:107BA00004D129002000FEF727F976BD012210211B
:107BB000200000F047FE0028F3D0F6E7014B1860E4
:107BC0007047C0464866FF1F37B56B469D1D0100D4
:107BD00004000222280003F02FFE2B88B02B0ED1C8
:107BE0002379122B09D12300FF339B78012B06D177
:107BF0000121608800F0E0F801E01B2BF8D037BDD0
:107C000010B5054B0421187000F098F8FFF74CFDF3
:107C1000FEF770FB10BDC0464C66FF1F0020F0B59C
:107C20000BB20F0087B0834234DA274B187803F089
:107C300043FC051E2BD00378A02B25D103AE3100C9
:107C4000FEF7E4F8041E0BD1B378DB0724D51F4BF5
:107C500006341B68002B03D0310068889847040065
:107C6000A868002801D003F0EFFE002C08D1184AC4
:107C7000039B1340174A934206D0B3781B2B03D0C3
:107C80000121688800F098F8280003F0ADFC8020FE
:107C90000002784007B0F0BD0F4B1B68002B10D0DE
:107CA000310068889847041EDAD07378002BD7D14A
:107CB000B27801A90A704B800C716888FDF7F6FF55
:107CC000CEE70624F1E7C0464C66FF1F4466FF1F5F
:107CD00000FFFF00000112004866FF1FF7B501908A
:107CE000822040000D0017001E0003F0E5FE040096
:107CF0001320002C12D0B02320002370089BFC22FC
:107D00006770658026710830002B08D0190003F0D9
:107D10007BFE2100019803F057FE0020FEBD08996C
:107D200003F0AAFEF5E710B5041E06D00078FD2882
:107D300003D803F089FDFF23237010BD0A1F93B2FF
:107D400010B504000220032B05D882400020024B0E
:107D5000D1529B189C7010BD6C66FF1F0B8870B5CC
:107D6000043B04000D000220032B0BD8012120004E
:107D700000F04CFD03001420002B03D0290020004C
:107D800000F0DEFB70BD000007B51300034A00924F
:107D90000A00012100F02CFC0EBDC046C57F001179
:107DA00007B5019203220092024B0A00122100F053
:107DB00049FC0EBD4380001107B56B4601AA118036
:107DC0000449D88008780633012802D1190003F04D
:107DD000E3FC07BD4D66FF1F0C4B10B51870002368
:107DE000FF210B4A1380138193819380094A5380AA
:107DF0001370517293819372D174D382137551773A
:107E000003F042FD00F0FCF910BDC0467C66FF1F88
:107E10006C66FF1F4E66FF1FF0B58DB06B460020ED
:107E200003910C229B5E834200DBB0E05D4B18782F
:107E300003F042FB051E00D1A4E00378902B00D094
:107E40009DE006AF01004688380000F013FA79681B
:107E50000400002900D19CE03B88052B6ED13B89B2
:107E6000032B1CD905AC200000F0A2F86288172A69
:107E700061D83989131D994231D179682378043149
:107E80000291D90738D5607800F08EF9071E06D028
:107E9000002303712378012B08D0132B23D0A8686B
:107EA000002800D178E003F0CFFD75E062880299E8
:107EB00009A800F0A6F80290380000F08BF909AA92
:107EC0002378387A0192002231000092029A00F061
:107ED00012F9380000F064F9029B002BDFD030006B
:107EE00000F080F9DBE70378032BD8D16288029990
:107EF00009A800F0D6F8DEE7122B13D1029909A8E1
:107F000000F0B5F8021EEAD127498B88002BC6D0B5
:107F1000887909A92378019161780091310000F0F6
:107F2000EAF8BCE7002302AA93833000617809AA2B
:107F3000FFF72AFFB3E71D4B0993F6E7042B02D0A6
:107F40009A1F012AABD8184A043B9B00995A002972
:107F5000A5D0D218907831003A0000F0AEF8002891
:107F60009DD13B88042B03D001213000FFF724FF73
:107F7000012C04D1A868002801D003F065FD280079
:107F800003F032FB8020039B0002434018000DB039
:107F9000F0BD012800D182E701213000FFF70CFF7E
:107FA000EDE7C0467C66FF1F6C66FF1F01001700EF
:107FB0000B7803704B784370CB788A781B0213439D
:107FC000438070470A88030002700A88120A4270D0
:107FD0000A88012A06D14A8882704A88120AC27029
:107FE0000420704702208242FBD14A8804309A70F4
:107FF0004A88120ADA708A881A718A88120A5A71B3
:10800000EFE710B50400012082420CD94B780A78C2
:108010001B0213432380834206D1CB788A781B024C
:1080200013436380002010BD022BFBD1CB788A78EC
:108030001B02134363804B790A791B021343A3800D
:10804000F0E70B8803700B881B0A43704B88837022
:108050004B881B0AC3708B8803718B881B0A437182
:10806000CB888371CB881B0AC3710820704703003B
:108070000120082A14D14A780878120202431A8093
:10808000CA788878120202435A804A790879120223
:1080900002439A80CA798879120202430020DA806A
:1080A000704710B504000120022A05D100204B784A
:1080B0000A781B021343238010BDF8B50600102078
:1080C0000F00150003F0F8FC04000120002C0ED076
:1080D000A0230C22290023806780201D002D07D0BB
:1080E00003F092FC2100300003F06EFC0020F8BD8C
:1080F00003F0C2FCF6E7F7B51E00009008AB1420B1
:1081000017001D78019103F0D7FC041E12D0A223A2
:108110000370019B47704380099B057146710C22D7
:108120000830002B07D0190003F06EFC21000098E6
:1081300003F04AFCF7BD099903F09EFCF6E737B55A
:10814000041E0FD04388002B0CD00025C1881323B8
:10815000007A172201950095FFF7CDFFFF23658078
:108160006372257037BD000010B50C4904004A88C1
:10817000002A09D08B89002B05D00020CB8A02224F
:10818000834201D010BD012213000A204343002086
:108190004032C854C81842800472F3E74E66FF1F8D
:1081A0000023438003707047094B00211A0010B56B
:1081B0005C88002C06D01C79844203D10A234B43EF
:1081C000D01810BD01310A330329F1D10020F8E79E
:1081D0004E66FF1F10B50400407A03F035FBFF2305
:1081E000637210BD7047043010B580B203F0CCFA52
:1081F000002803D00421494203F0F6FA10BD000024
:1082000070B50025104CA0682580A581A580A842E6
:1082100002D003F019FCA56000250C4C0C4B606DDE
:108220001D80230058331D70A84202D003F00CFCBF
:10823000656500256068002801D003F005FC013564
:1082400008340A2DF6D170BD1467FF1FB866FF1FF2
:108250000867FF1F70B5041E09D1054D2880A8814D
:10826000A880A868002802D003F0EEFBAC6070BDC7
:108270001467FF1FF0B54B8885B00193002343605E
:108280000A7905000F00022A00D07BE0CA88032A81
:1082900017D98B685E7819783602DC78D8790E4366
:1082A00099781B7A24021B020C43034353495BBA9F
:1082B0000B80331D93421ED1042C04D0631F022B6C
:1082C0000ED9012015E0019A4D4B1201D35A002B13
:1082D00006D00198FFF7BEFF4A4A136901331361C4
:1082E0000421B8682E812C80494203F07DFA686031
:1082F000002005B0F0BD434D042C06D0631F022BB7
:108300000FD9EB680133EB60DBE7019A3C4B1201BC
:10831000D35A002B05D00198FFF79CFF2B6901333E
:108320002B61374B30000293019B029A1B01019392
:10833000002301998C468B52130063449C80039365
:108340009E81FFF750FF039B041E986016D0042106
:10835000B868494203F048FAFA880100043A20005C
:1083600003F052FB0199029AFB888A5A043B9B183E
:10837000029A8B522B6801332B60A2E7AB69013361
:10838000AB619EE71E4B0293019B1E01029BF35AB9
:10839000002B2DD002998C19A068002828D0012A22
:1083A00026D1FA889B189BB27352A189994217D3A0
:1083B0009B1AC018B96803F027FB029BA289F35AE5
:1083C000934200D07DE700222B81A3882B80A368F5
:1083D0006B60029BF2520B4A53680133536070E7A3
:1083E000084A9368013393600198FFF733FF68E709
:1083F000044A536901335361F6E7C0467E66FF1FA6
:108400001467FF1F8466FF1F70B5051E15D10B4C46
:108410000B4B1880230058331870606D002802D071
:1084200003F012FB6565250050356068002801D017
:1084300003F00AFB0834AC42F7D170BDB866FF1FE9
:108440000867FF1FF0B51700A12285B092000193C5
:108450004243394B06001B680C009B18D933FF338D
:108460001D78FDF741FF0430854204DD3000FDF743
:108470003BFF0430C5B2BD4207D33A0000213000B3
:10848000019B03F0A1F905B0F0BD2900380003F00D
:108490005BFA2300C6B250331E700393019B290080
:1084A0006365380003F0E0FACBB20293002B02D0F0
:1084B000039B01361E7000262300503303931B7864
:1084C000B34204D8606D002831D10020DBE7029A66
:1084D0002800002A04D0013B1000B34200D028003D
:1084E000F700E719387003F03FF8786000280ED0E5
:1084F0003A78019903F088FA019A3B780136D3184B
:108500000E4A0193D369F6B20133D361D4E7039BDA
:1085100018706065A74205D1084A1320D36A013359
:10852000D362B0E7606803F08FFA0834F2E703F033
:108530008BFA00236365C8E73409FF1F8466FF1FB9
:10854000F7B50D0007000421686803F04DF92B8989
:10855000040003702B891B0A43702B8883702B88BF
:108560001B0AC3702E8902250436F6B2FB2E15D8DD
:108570001B4B9F4214D10C2003F09EFA1135011EB3
:108580000CD0902303708E3B0371043B4380154B4A
:108590008460C680187803F017FA00252800FEBD15
:1085A0005C237B43104AD3180093583301931B7804
:1085B000002B0FD10300320038000099FFF742FF73
:1085C000019B05001B78002BE8D13800009902F0D0
:1085D0007BFFE3E7054A0725536A01335362DDE772
:1085E000FEFF00007C66FF1FB866FF1F8466FF1F4A
:1085F000F0B587B0009017200F0016000193FFF729
:10860000F2FD1325041E19D00C98031E02D0019907
:10861000201D9847030AE370052302AAA0700430C6
:10862000908127700098667003A993800494FFF7E7
:1086300087FF051E02D0200003F006FA280007B0CD
:10864000F0BD0000F0B587B01F000CAB1B780391A4
:10865000059301210DAB06001C78049200F0D6F8BA
:108660001425002821D02000FFF77EFD0135041ECF
:108670001BD01149059B0A7803700132D2B2131E38
:10868000C68001D101231A000B7022713000049BB7
:1086900003990097FFF7ACFF051E09D123002100C5
:1086A0000648074A093302F02FFF280007B0F0BD43
:1086B000002363802370F8E78066FF1F3F8100116D
:1086C00030750000F8B505000E00064C064F236813
:1086D000002B02D03100280098470434BC42F6D168
:1086E000F8BDC0462467FF1F3867FF1F0123064AF5
:1086F0005B425380002313715362044A136053603A
:108700009360D360136170473867FF1F2467FF1FB2
:108710000200002310B506499C000859002801D129
:10872000625010BD0133052BF6D11320F9E7C04686
:108730002467FF1F034A5388181A43425841404296
:10874000104070473867FF1FF0B585B002930AAB41
:108750001F780CAB1B88009008000E000192039359
:10876000FFF7E8FF05001120002D1BD10E48FFF791
:10877000E1FF04001520002C14D006220B99A771EC
:10878000E01D03F041F9019B30002371029B290099
:108790006371009B66802370039B6562E381FFF732
:1087A00091FF280005B0F0BDFFFF000010B5FFF7F6
:1087B000C1FF04000220002C12D060880121FFF7C5
:1087C00081FF606A002801D002F016FF28220021F4
:1087D000200003F051F9012300205B4263802071E7
:1087E00010BD000030B5074A074C558801001378CA
:1087F0000020A54204D05B1A59424B415842104018
:1088000030BDC0463867FF1FFFFF0000084A10B5A3
:1088100001230C00904208D0FFF78CFF031E04D008
:10882000037923405A1E9341DBB2180010BDC046A5
:10883000FEFF0000024B1879431E9841C0B27047FA
:108840003867FF1F70B504000D001600FFF772FFB8
:10885000002804D10D4B9C4200D0143070BD416AF9
:1088600003790520002907D012221A40102A02D1CC
:108870000520002EF2D10F20DB06EFD5897E0C20DB
:10888000A9428941494249420840E7E7FEFF00000A
:10889000030010B5002800D110BD0348034A4188E9
:1088A0009142F9D09847F7E73867FF1FFFFF0000B4
:1088B000002330B5C45CCD5C6C40D4540133102B24
:1088C000F8D130BD0F23002210B5C45C64002243F0
:1088D000CA54C25CD209013BF7D210BD02000100AC
:1088E00010B52032103102F027FF10BDF0B58BB06B
:1088F0000390102005931700049103F05DF8009099
:10890000102003F059F8009B13240190002B05D090
:1089100000280CD11324009802F06EFE019B002B5E
:1089200002D0180002F068FE20000BB0F0BD10204D
:1089300003F042F80600102003F03EF8132405006F
:10894000002E00D1AEE0002819D01022002103F043
:1089500093F832002900039802F0EEFE041E0ED1B7
:1089600033787F2B51D830000099FFF7ABFF009B85
:108970001B787F2B53D801990098FFF7A3FF300095
:1089800002F03AFE002D02D0280002F035FE002C45
:10899000C1D1102003F010F80600102003F00CF8ED
:1089A0000290002E7CD0002878D03A000F322300AD
:1089B0000125121105D00F333B4015B25A425341E5
:1089C0001BB26A1E1201002B33D0049BD2B298183E
:1089D0000099029AFFF76CFF013D10220021300040
:1089E00003F04AF8ADB2049F2D017D19AF4242D089
:1089F000002C33D0300002F0FFFD029B002B00D191
:108A000089E7180002F0F8FD85E729003000FFF73C
:108A100059FF28002549009AFFF74AFFA7E72900D8
:108A20000098FFF74FFF28002049019AFFF740FF09
:108A3000A5E70F210F4004998A18D9B28F4208D9AF
:108A4000D15C06A819540133102BF6D1029A019972
:108A5000C0E7791A48424141C901F2E739003000C4
:108A600006AAFFF725FF3200039806A902F064FE6C
:108A700010370400BAE7002CBCD13000029906AAD6
:108A8000FFF716FF320006A9039802F055FE0822F0
:108A900004003100059802F0B7FFABE71324A9E703
:108AA0001324AAE7002800D06EE733E760BD001169
:108AB000F0B58BB00F0016000225009000283FD0C3
:108AC000002A3DD00B1DDBB21800029302F074FFA8
:108AD0001135041E34D0FDF747FD05003A0000991A
:108AE000201D02F079FEEBB20393E3702B0CDBB296
:108AF0002F0A00936370FFB22B0E2370A7700193AF
:108B0000FDF72CFD1022010006A802F065FE2100F1
:108B1000029A04AB06A8FFF7E9FE051E0DD1039BE0
:108B200008223370009B04A9B370019B7770F37027
:108B3000301D02F051FEFDF71DFD200002F05CFD2E
:108B400028000BB0F0BDF0B58FB00D00149E03905F
:108B500004920593002A03D1022420000FB0F0BD37
:108B6000002EF9D00398FFF7E5FD1424071EF4D07A
:108B70007278337812021A43B3781B041343F278E5
:108B800012061A43036A0192934201D30133E3D1DF
:108B9000002D03D03B7901249B07DED5082200215C
:108BA00006A802F069FF059B13240433DBB218000A
:108BB000029302F001FF051ECFD0059A04990430FC
:108BC00002F00AFE04223100280002F005FE3900FE
:108BD000102210310AA802F0FFFD2900029A06AB0C
:108BE0000AA8FFF783FE041E0FD1082206A908A8D1
:108BF00002F0F2FD0822311D08A802F07DFC0128D8
:108C000007D101990398FDF7C9FC280002F0F4FC94
:108C1000A3E70124F9E7000070B51C4C05002368A8
:108C2000181E10D0002D14D11A78002A0CD1981CCF
:108C3000083202F0E9FE02F09FFC0135002808D15D
:108C400023681D70012070BD0A331800082202F04D
:108C5000DBFE2368002BF5D0122002F02DFF061E4C
:108C60000DD0C123216803704570023110220230FB
:108C700002F0CAFE23683100587802F0A5FE206891
:108C800002F0BAFC00232360DCE7C0466067FF1FE8
:108C9000F8B504002020FDF755FB0D4EA700BB5989
:108CA0000500002B0DD000280BD0D878FF2809D163
:108CB00008492A000C55F35907480333611802F09C
:108CC00023FCF8BD290002F0C7FD0028F0D1F8E729
:108CD0007C67FF1F6467FF1FE99E001170B5064D9A
:108CE00084006359002B05D0D87802F0ADFDFF2237
:108CF0006359DA7070BDC0467C67FF1F70B506000F
:108D00008CB00C00150000213022684602F0B4FE41
:108D100031001022684602F05FFD1D202100032271
:108D2000684402F059FD6846FFF7D8FD2D21040084
:108D300003222800694402F04FFD20000CB070BDF2
:108D4000F0B50700160097B001931CAB1D783022D8
:108D50001EAB00910AA800211C7802F08DFE1022A3
:108D600039000AA802F038FD1022002102A802F002
:108D700083FE0722310002A802F02EFD072202AB7B
:108D80009818631E9C41019902F026FD02AB9C736A
:108D90002B005A1E934102AAD3730021102206A869
:108DA00002F06AFE06221D9907A802F015FD1A209E
:108DB00002ABC01806221F9902F00EFD1022009986
:108DC0000EA802F009FD102202AB0EA908781C784B
:108DD000013A6040D2B2087001330131002AF5D166
:108DE0000AA8FFF77BFD102212A904000EA802F0CA
:108DF0000BFE102206AB0EA908781D78013A6840D8
:108E0000D2B2087001330131002AF5D10AA8FFF768
:108E100065FD044310222098E4B212A902F0DCFCA4
:108E2000200017B0F0BD70B50E0014008CB001002A
:108E3000102268461D0002F0CFFC3100082204A871
:108E400002F0CAFC2100082206A802F0C5FC684610
:108E5000FFF744FD04001022280008A902F0BCFC22
:108E600020000CB070BDF8B506000D0000243719C5
:108E7000AC4200D3F8BD02F03FFD030A3B70631C17
:108E8000DBB201379D4203D90234F054E4B2EEE77D
:108E90001C00EDE773B506000C000225002819D070
:108EA000002917D0032101A8FFF7DDFF6B469A794F
:108EB0003F231A40013313436A463000937101A9DE
:108EC0002200FFF71BFF051E04D10322E01C01A9AD
:108ED00002F09AFD280076BD03785807DA08C00F23
:108EE000D20080009B0710439B0F1843C0B270470D
:108EF00007230B40C908C9000B43037070470000EB
:108F000070B50400FFF7EAFE134DA4006359002B6F
:108F100021D0186A002801D002F06EFB2B59986E00
:108F2000002801D002F068FB2B59D86E002801D030
:108F300002F062FB2B59186F002801D002F05CFB95
:108F40002B59586F002801D002F056FB285902F027
:108F500053FB00232B5170BD7C67FF1F0E4B80001D
:108F6000C35870B50C00002B0FD09D68002D0CD09D
:108F70002B78201D0B706B784B70A97CFFF7B8FF26
:108F80002B7E23726B69E36070BD102200212000EC
:108F900002F072FDF8E7C0467C67FF1F014B1860C6
:108FA0007047C0467867FF1F074A03008000825859
:108FB00010B5002A06D0D088984203D1012901D1EA
:108FC000FFF79EFF10BDC0467C67FF1FF0B5264E21
:108FD00095B087000B93BB590500099112200A92A6
:108FE000002B31D0D888FFF7A5FB04001420002CFB
:108FF0002AD0280010A9FFF7B1FFBB591E781D6ABF
:10900000002E23D00895FDF7EFFA07000020FDF7AA
:10901000F1FA0790A379E61D069310AD0CA9089804
:1090200000F0E2FA0EA9280000F0D7FA0B9B0A998B
:109030000493069B09980293079B0396019300975C
:109040000EAB0CAAFFF77CFE15B0F0BDFDF7CCFA15
:1090500006903000FDF7CEFAE31DA779079310AB19
:1090600006000893DAE7C0467C67FF1F30B50C4C5A
:1090700085002A59030085B00120002A0ED018006F
:109080006946FFF76BFF2B591A78D888054B002AE1
:1090900000D1054B6A46072100F0D9FB05B030BD71
:1090A0007C67FF1FDB950011E995001130B5094C75
:1090B0008500295985B010226846253102F0A4FCAC
:1090C0002A591121044BD0886A4600F0C0FB05B034
:1090D00030BDC0467C67FF1F8596001130B5094C36
:1090E0008500295985B010226846353102F08CFC84
:1090F0002A591121044BD0886A4600F0A8FB05B01C
:1091000030BDC0467C67FF1FC3960011F7B54D4FB9
:1091100086001020F4590D0002F04EFCF359206235
:10912000186A132200286CD0033A29009C6802F0C8
:109130006BFCF3591A780192002A58D11E6A227DDD
:10914000317B944651400122019F114201D1674673
:109150001740217D914339432175377B4F40BC46F1
:1091600060460027800701D44F08174001210220E4
:109170008F40227D82433A432275377B5740BC465D
:1091800060460027400701D497080F400420227D45
:10919000BF0082433A432275627D002794466046B1
:1091A000727B42400A4201D167460F400121627D35
:1091B0008A433A436275777B5740BC466046002736
:1091C000800701D457080F400220627D7F00824350
:1091D00017436775767B00227E40760701D4BA0874
:1091E0000A400426617D9200B1430A4362756A78A1
:1091F000002A08D06278002A05D005220533DA77E4
:1092000000221000FEBD04222979114205D1A17C63
:10921000114202D10533033AF1E7019A21782C7803
:10922000002A02D10A002100140018220429E8D8DB
:10923000042CE6D805206043034A05331218525C1B
:10924000DDE7C0467C67FF1F70BD001110B50A0046
:109250001121024B00F0FBFA10BDC0461F97001110
:109260000B0030B587B001AD2B806B4604001100B8
:10927000981D082202F0C8FB2A000B212000024B97
:1092800000F0E5FA07B030BD4797001110B50A00AD
:109290001121024B00F0DBFA10BDC0469B97001174
:1092A00013B50B0011006A4613706B4604000622CA
:1092B000581C02F0A9FB6A4608212000014B00F06F
:1092C000C6FA13BDBB97001110B50A001121024B5D
:1092D00000F0BDFA10BDC0460B9800117FB5050027
:1092E0000B4BAA00D4580800002C0FD0666F237FC8
:1092F000E28821780396266F0296E66E0196A46EA8
:109300000094FDF709FC2800FFF7FAFD7FBDC04679
:109310007C67FF1F10B51721FFF7E0FF10BD0000AD
:1093200070B50A000D00064B0221040000F08FFA10
:10933000060029782000FFF7D1FF300070BDC0463D
:10934000EB96001170B586B000236A4613708368EF
:1093500004001D78681E0A2859D801A902F014F9E2
:10936000060633373B3F43474B4F5300180000F08E
:1093700042F9062312284BD000281BD16088FFF742
:10938000D9F90823002813D04279002A47D1264B67
:109390001A78072312070BD5244B1A680723002AD3
:1093A00006D01668002E03D0290001AAB04703009A
:1093B0006A4613706B461B786088002B2AD1FFF732
:1093C00067FC06B070BD180000F06CF9D4E7180017
:1093D00000F087F9D0E7180000F093F9CCE7180007
:1093E00000F0ADF9C8E7180000F0C3F9C4E71800B1
:1093F00000F0F6F9C0E7180000F0F6F9BCE7180035
:1094000000F013FAB8E7180000F013FAB4E70723E6
:109410006A46137069466088FFF782FFD1E705232B
:10942000012AC5D1024BB8E70966FF1F7467FF1F09
:109430007867FF1FF8B52C4F8600F35904000D0024
:10944000002B40D0DA8882423DD15A78062A33D1A7
:109450001A78002A2ED0012099681A6A097D0142E3
:1094600006D0157B054203D007225A700120F8BDB3
:109470000220014204D0157B054201D00922F4E705
:109480000420014204D0127B024201D00B22ECE7FF
:10949000164B1B68002BE9D05B68002BE6D0200040
:1094A0009847BB5900215B78122BDFD12000FFF7D2
:1094B00015FFDBE70E4BECE7112A04D1002900D0A1
:1094C00032252900F2E7002D08D12000FFF732F9FC
:1094D000002803D0102302791343037121002800D0
:1094E000FDF798FAC2E7C0467C67FF1F7467FF1F4D
:1094F0007867FF1F70B50E4E8500AB590400002B36
:1095000013D01B78002B11D10A4B1B68002B04D001
:109510005B68002B01D02000984773595B78122BB1
:1095200003D100212000FFF7D9FE70BD024BECE70C
:109530007C67FF1F7867FF1F7467FF1F094B800060
:10954000C3581020002B0CD01A6A002A09D09B683F
:10955000002B06D0127A1B7E101C9A4200D9181CD0
:10956000C0B270477C67FF1F70B503000D00140088
:109570000220002A30D000292ED013700B78081D4D
:1095800053704B789370FFF7A7FCE0700120022125
:109590002B7A23716B7B034063716A7B0A40134310
:1095A000042263716E7B1640334363716E7BF60851
:1095B000F600334363712B7B0340A371287B01408A
:1095C00000200B43A371297B0A401343A3712A7B1C
:1095D000D208D2001343A37170BD10B50A00010078
:1095E0000120FFF7C1FF10BD10B50A0001000220E5
:1095F000FFF7BAFF10BD70B506000C000220002E68
:1096000030D000292ED07378201D0B70B3784B70AA
:10961000F178FFF76DFC01223579257271794B10D5
:10962000080013409340104003438810104080000E
:10963000C9080343C9000B436373B1794B10080099
:109640001340934010400343881002409200C90821
:109650001343C9000B4321202373FCF773FE85429B
:1096600001D2122070BD2220257AFCF76BFE8542C4
:10967000F7D823781820042BF4D86378012BF1D87D
:109680000020EFE7030010B50220002909D0002BCD
:1096900007D00322481C0A7019000D3202F0B4F9F9
:1096A000002010BD03000222080010B5002B06D0D8
:1096B000002904D00E32591C02F0A6F90022100035
:1096C00010BD030010B50220002909D0002B07D0DF
:1096D0000422481C0A7019000C3202F095F900208F
:1096E00010BD10B5FFF7DEFF10BD030002200029FA
:1096F00006D0002B04D0052200200A701B784B7086
:10970000704703000220002B08D0002906D05B78A8
:1097100000200B70013B082B00D918307047030064
:1097200010B50220002909D0002B07D00622481CC2
:109730000A7019000A3202F067F9002010BD10B556
:10974000FFF7B0FF10BD02000B00022010B500298A
:109750000ED0002A0CD00721197011885970118879
:10976000090A997011180822D81C02F04DF900203E
:1097700010BD03000A00022010B5002B0CD00029F8
:109780000AD099785878090201431180901CD91C9D
:10979000082202F039F9002010BD030010B50220A4
:1097A000002909D0002B07D00822481C0A70190094
:1097B000921802F029F9002010BD02000B000220CF
:1097C00010B500290BD0002A09D009211970117891
:1097D00018185970511C062202F016F9002010BD0D
:1097E00010B5FFF75FFF10BD02000B00022010B59F
:1097F000002A09D0002907D05178197011180622C3
:10980000581C02F001F9002010BD030010B5022021
:10981000002909D0002B07D00A22481C0A70190021
:10982000063202F0F1F8002010BD10B5FFF73AFF44
:1098300010BD02000B00022010B5002A06D000293E
:1098400004D018005178FFF753FB002010BDF0B58D
:1098500085B017001E006A460623050008009181A6
:109860009380FEF7C0FC1324011E02900CD0380038
:10987000B047041E05D1280001A9FEF76FFA041EA7
:1098800002D0029802F0E0F82800FFF701FA200069
:1098900005B0F0BDF0B504008BB0019115000021BA
:1098A000102202A802F0E8F8334EA700B8590028A9
:1098B0003CD0C388A34239D10378002B36D14278FB
:1098C000062A18D102000100553235310C3006ABA2
:1098D000FFF7A9FA002829D12000FFF72FFE020088
:1098E00006A902A802F090F8200002A901F034FEB7
:1098F00001200BB0F0BD816E002917D00B8A112A10
:1099000028D19D420ED101981231093A01F0F4FD9F
:10991000012807D1BB5920009D6EFFF70FFE2900DB
:109920000200DEE732212000FFF7D8FC2000FEF71E
:1099300001FF061E1BD0416A002918D00B8AAB42DA
:1099400015D108220198123101F0D6FD01280ED15F
:10995000716A0AE09D42E9D108220198123101F0B2
:10996000CBFD0128E2D1BB59996E8A7EB9E7200070
:1099700001F042FFBCE7C0467C67FF1FF0B56B4DAE
:1099800087007E5985B0337802900393002B00D076
:1099900087E0B368346A01937078062817D10122F2
:1099A0001B7D134202D0217B114218D102221342A7
:1099B00002D0217B114251D10422134203D0237BD8
:1099C000134200D08BE0019B5A7DEB5991E00738A0
:1099D0000428F8D801F0D8FD032E42678300B36E47
:1099E000002B03D11C2001F0E7FFB066EB599C6E01
:1099F000002C1CD010220021200002F03DF802981B
:109A0000FFF79CFD01002000FFF72DFA01F074FF25
:109A10002082200008211230FFF725FA0298FFF774
:109A20008DFDA076EB592100D888FFF70FFC0822A6
:109A3000EB591CE0B36E002B05D01A00198AF08890
:109A40001232FFF70DFC0222019B197DEB591142E6
:109A50003DD0207B10423AD0073208E0F488FCF772
:109A6000DBFD01002000FFF711FC0A22EB595A70C0
:109A7000029B9C002A595378073B042B11D8D088AD
:109A8000FEF758FE00284ED0C3895A08D21828493C
:109A9000029B0298CB542B5941180433254801F0FE
:109AA00033FD05B0F0BDFCF79FFD030001208342AC
:109AB00001D100200393EB59DE88FCF79BFD03994D
:109AC00002003000FFF7ECFB019AEB59117D0422F4
:109AD00011420CD0217B114209D00B22C7E7F68836
:109AE000FCF73CFD01003000FFF7EEFB6BE7019A4D
:109AF000527D01210A4204D0607B084201D00C2231
:109B0000B5E702210A4204D0607B084201D00E2250
:109B1000ADE704210A4204D0627B0A4201D0102240
:109B2000A5E71222A3E7FA225200B0E77C67FF1FE5
:109B30008067FF1FF39E001110B5064B1A780423AF
:109B4000100018401A4200D00348FFF727FA0020FF
:109B500010BDC0460966FF1F8C44FF1F70B504008E
:109B6000FFF7D4FA051E43D12000FFF77FFA234EFA
:109B7000A400A0598268937CDB0708D50321036AFF
:109B80001B790B40012B02D1017F0B430377431D4F
:109B9000D97F8B1E022B0DD8022900D00121C0884D
:109BA000FCF790FF042133591A7F59700A431A7742
:109BB000280070BD01290CD102231022437000211E
:109BC0000C3001F059FF305910213530FFF74BF9B7
:109BD000EEE70529ECD10223D118437010220C3096
:109BE00001F012FF04233259117F0B431377EAE788
:109BF00008251828DCD1053DDAE7C0467C67FF1F41
:109C0000F0B58BB0059143887E4F9E00F459150046
:109C10000493002C15D1012902D000200BB0F0BD17
:109C2000101D57781678FFF757F9EB68320002934A
:109C30002B7A0499019300903B002000FCF70CFF65
:109C4000EBE7E388049A934201D00820E6E7237803
:109C5000012B00D1D4E0059B581E092800D9CFE084
:109C600001F092FC05CE0A29CC506C859AB22900ED
:109C70000498FFF773FFD1E7200029001022453038
:109C800001F0C2FEB9594B78042B02D1013B4B7055
:109C9000C3E70B000A00253335320C310498FFF777
:109CA00095F90498FFF702FA0522431E9841BB5923
:109CB000C0005A70B2E7200029001022553001F090
:109CC000A3FE049B4F4C9D00295904980A0006AB43
:109CD00055320C31FFF77AF929591022453106A87F
:109CE00001F00AFC012808D10498FFF7F7F9059064
:109CF000002804D106222B595A7005988EE70823B4
:109D00000593FAE763780C2B7AD1E36E002B03D12D
:109D10001C2001F051FEE066BB59D86E00286FD0C0
:109D20001022290001F070FEBB590498DC6EFFF789
:109D300005FC0D22A076BB595A706EE7E06E002834
:109D40005ED063780D2B5BD12B8808220382A91C7F
:109D5000123001F059FEBB599A68517D022211421E
:109D600026D0186A407B104222D00C32E4E7637898
:109D70000E2B45D1236F002B03D1162001F01CFEC2
:109D80002067BB59186F002803D01022290001F06A
:109D90003BFE0F22BB59CFE763780F2B30D1206FEA
:109DA0000622691C103001F02FFEBB599A68517DC4
:109DB0000422114203D0196A497B1142D5D10021F6
:109DC0000498FFF78BFA28E7636F002B0DD0BB597F
:109DD000586F0028F3D01022290001F015FE01224F
:109DE000BB5952425B6F1A61E9E7142001F0E4FDB0
:109DF000BB5960675B6F002BE9D126E72978DFE765
:109E000007200BE77C67FF1F10B5064C207001F0A0
:109E1000DBFB06212078FDF791FF0348FEF778FC75
:109E200010BDC0468F67FF1FA98F001100200BB225
:109E300070B50D00834216DA264B187801F03CFB12
:109E4000041E0DD00378922B0ED0A02B37D0224BBE
:109E50001878FF283AD0210001F0B6FD002835D14E
:109E600080200002684070BD43780E2B0BD03E2B43
:109E7000EDD18378052B12D0082BE8D18179808829
:109E8000FFF7D8FA08E0154B82889A42DFD1836841
:109E90001878591CFEF7C0FE002817D1D7E7104BE1
:109EA0001B785B0712D50F4B1B68002B0ED09B68ED
:109EB000002B0BD0C289811D80889847ECE7FFF703
:109EC00041FAA068002801D001F0BEFD200001F099
:109ED0008BFBC5E78F67FF1F8544FF1F182000001D
:109EE0000966FF1F7867FF1F10B50078FFF712FAA9
:109EF00010BD10B50078FFF7FDFA10BD0C234343E9
:109F0000084A10B59B185A68002A03D0012901D1CC
:109F1000904710BD9B68002BFBD00029F9D19847D2
:109F2000F7E7C046AC67FF1F10B5162813D801230A
:109F30008340094A946B1C439463506B984350636D
:109F4000D46B20009843012901D120001843D0632D
:109F5000116B0B43136310BD00800040F0B500246B
:109F60000127154B85B0DA6B144E03921A6C0192DF
:109F7000DA64019BE3403B4217D0039DE5403D403E
:109F80000295E5B202992800FFF7B8FF316A736ABB
:109F9000002908D03900002B01D00299794028000F
:109FA000FFF7C2FF01E0002BF9D101340C36172C6A
:109FB000DFD105B0F0BDC046008000409067FF1FB4
:109FC00010B5012402002000162A08D8054B596854
:109FD000D140214204D01868D0400123184010BD60
:109FE000186DF9E700800040162807D80122064BBB
:109FF0008240002903D0D9680A43DA607047D968E3
:10A000009143D960FAE7C0460038004030B51628C1
:10A0100018D8032444430F4BE25C1B199C785D78ED
:10A0200001232D1B0135AB40013BA340A140DB4385
:10A030000C00122807D808499200521811681940DC
:10A040002143116030BD054A11680B402343136062
:10A05000F8E7C046B7BD001108F0004014F000401A
:10A06000C21F70B5D4B20623092C0BD80125084CA9
:10A070009540002908D00021FFF7C8FF23682B4333
:10A0800023600023180070BD2368AB43F8E7C04687
:10A0900000380040F0B5162826D8214B1B185B78F5
:10A0A000022B21D1032444431E4A1F4EA35C1219E4
:10A0B0009478012215008540B76B013CE4B23D4322
:10A0C000A240B563194C122815D89B0000290CD169
:10A0D00017495B1899680A439A600123205C154A66
:10A0E000834011680B431360F0BD11495B189968F8
:10A0F00091439960F1E70E4B00290DD159690A434C
:10A100005A61225C1328E8D00123203A93400A497F
:10A11000086803430B60E7E7596991435961F0E729
:10A120009067FF1FB7BD001100800040FCBD00110B
:10A1300000F00040A0F00040A4F00040F8B500247A
:10A140001B4E1C4D1C4B1B5D012B1FD1184A9269E5
:10A15000E2401A420BD00122AA5693402200143A40
:10A16000D2B2022A09D815494A6913434B61013416
:10A170000C360235172CE5D1F8BD0022AA560F493E
:10A180009200521891680B439360F0E7022BEED1D6
:10A19000E7B23800FFF714FF01235840C1B238007E
:10A1A000FFF778FF3800FFF70BFF7077DFE7C04657
:10A1B0009067FF1F89BD00119167FF1F00F00040ED
:10A1C000012202388240054B002903D059690A4315
:10A1D0005A617047596991435961FAE70038004064
:10A1E00070B504000D000520162C1AD8002120009F
:10A1F000FFF7FAFEA31E012B03D801212000FFF771
:10A20000DFFF00212000FFF72BFF01220A49A240B7
:10A210000A4B4868012D05D102431B194A605D7045
:10A22000002070BD9043486002211C19617099693B
:10A2300091439961F4E7C046008000409067FF1F9A
:10A2400010B516280AD80122074B8240002906D0F3
:10A2500019680A431A600121FFF7C2FF10BD19688F
:10A2600091431960F7E7C0460080004070B50500D3
:10A270000520162D17D80C2300246B430A4A210011
:10A280009B181C70094B28005B195C70FFF7A8FF36
:10A290000123AB40200006490A681A430A600549B9
:10A2A0000A689A430A6070BDAC67FF1F9067FF1F82
:10A2B000348000403080004070B504000E00FF285C
:10A2C00013D003250540FFF7D1FF084AA3089B00E0
:10A2D0009B183F22ED00AA40AE4019682000914330
:10A2E000314319600121FFF77FFE70BD183800402F
:10A2F000F8B505000520162D25D80C246C43124B0B
:10A30000E4186368002B03D1A3680D30002B1AD02A
:10A31000022201270D4B00215B195A70280027707B
:10A32000FFF75EFF63681E1E08D0A3683E00002B87
:10A3300004D02800FFF744FE4640F6B22800310062
:10A34000FFF7F2FD0020F8BDAC67FF1F9067FF1F0D
:10A35000F7B5C420FF222B4B8000195800249143ED
:10A360007F3A0A431A508022274F5202274E1A6022
:10A37000274B1D5D002D21D0A31E012B03D80121E9
:10A38000E0B2FFF71DFF012D18D11F4B9B69E34081
:10A390002B4213D0E3B218000193FFF711FE010026
:10A3A0000198FFF74DFFE3B2143B022B1DD80121AA
:10A3B0007156184A8D405369AB4353613B7F002B64
:10A3C0000DD0E5B22800FFF793FF2800FFF7F8FD56
:10A3D0007B7F0100834202D02800FFF78FFD01340C
:10A3E0000C370236172CC3D1F7BD0121002371565B
:10A3F000F3568D40074A9B009B189A68AA439A60BF
:10A40000DCE7C04600E100E09067FF1F89BD001156
:10A410009167FF1F00F0004010B504000520162CC6
:10A420000CD801212000FFF7DBFE0123044A0020A5
:10A4300011194B70A34091690B43936110BDC04645
:10A440009067FF1F70B50E0015000400FFF70EFFA8
:10A450000C236343094A20009B189D605E60FFF750
:10A4600047FFF021064B074A8900051E5A5002D0CB
:10A470002000FFF7FBFE280070BDC046AC67FF1F41
:10A480000000FF1F5D9F001170B5134D07202C7851
:10A49000002C1FD1982221005200280001F0E4F97D
:10A4A0000123C420FF222B700C4B80001C635C63D3
:10A4B0000B4B1C605C600B4B195891437F3A0A436D
:10A4C0001A50802252021A600D20074A074901F0F3
:10A4D0000BFA200070BDC0469067FF1F008000404F
:10A4E000A0F0004000E100E051A300113DA10011E7
:10A4F000030010B50620072B09D8054A137000F099
:10A50000A3FFD7210020034B034A89005A5010BDF6
:10A51000B444FF1F0000FF1F151BFF1F70B51D0077
:10A5200002240C2910D8094ACA40D2070CD5FBF7DF
:10A5300015FF041E08D1059A04992800FBF72AFF8D
:10A54000FCF798FDFFF7F8FA200070BD121000002C
:10A5500030B50D7802232C009C43184201D02B43C8
:10A560001C0008252300AB43284201D02B002343C5
:10A5700020241D00A543204201D01C4325002A238E
:10A580000D70184204D011781E3B0B43137030BD80
:10A590000028FCD10C2113788B43F7E7F8B51D0098
:10A5A00006AB1B88140007AA0E000B201778002B9F
:10A5B00027D10A78022A49D14A68507811780002D6
:10A5C000244A08438018042840D800F0DDFF031215
:10A5D0001D1B2300F06801F0FFF9021CC0B2B84255
:10A5E00000D93A1CD2B22000F1682A8001F00CFA9E
:10A5F00006E00222F3681B882A8023701B0A63701E
:10A600000020F8BD0622EEE701232B80F3681B78BB
:10A610002370F5E7F368002B16D008222A801A88E9
:10A6200022701A88120A62705A88A2705A88120A16
:10A63000E2709A8822719A88120A6271DA88A2718D
:10A64000DB881B0AE371DBE72B80D9E701202B8035
:10A65000D7E7C04600D6FFFFF7B516000A781D0001
:10A6600008AB1F880C000123022A18D14A685078D1
:10A67000117800022B4A0843801803280FD800F0F5
:10A6800083FF02254439E06801F0A6F9C0B2072330
:10A69000B84204D37B190193152B02DD0D2318005A
:10A6A000FEBDE0682A003100C01901F0ADF96B462B
:10A6B00000209B88E268D0541B4B1B68834203D068
:10A6C0001B68834200D098470023E8E70B23002F44
:10A6D000E5D1022DE2D1737832781B021343E26890
:10A6E0001380114B1B68002BEED01B68002BEBD0A6
:10A6F0000120E8E70B23002FD1D1062DCED12A006F
:10A700003100E06801F080F9DEE70B23002FC6D1AD
:10A71000012DC3D132787533012AC0D8E3681A708D
:10A72000D2E7C04600D6FFFF9C69FF1F70B50C0042
:10A730001500072837D800F027FF041436361B36DB
:10A74000242E182015290BD8184E1622002130006F
:10A7500001F092F922002900300001F055F90020A3
:10A7600070BD18200229FBD11288114B1A80F6E720
:10A7700018200829F4D10A000E48290001F05CF8DD
:10A78000EDE718200129EBD10B4B10780B49DA6962
:10A79000FFF7DEFEE3E718200129E1D1064B107830
:10A7A0000749DA6BF4E70220DAE7C0468469FF1F45
:10A7B0003245FF1F2845FF1FB844FF1FE044FF1F1D
:10A7C0000045FF1F030010B50020DB0704D507215B
:10A7D000024A034800F08CF810BDC04614BE0011B8
:10A7E000B844FF1F054A03001068002803D0828880
:10A7F0009A4201D1806870470068F6E7A06BFF1F9E
:10A800000A88030008009A4204D08A8804309A42D9
:10A8100000D0002070470000F8B5F82200230D4F4B
:10A820000D4E7968050042433370994200D07B6039
:10A830000A4C0021200001F01FF900231A007C605F
:10A84000AB4202D100203370F8BD01332280DBB26D
:10A85000F834F5E7A06CFF1F9C6CFF1FA46BFF1F73
:10A8600073B56B4601900600684615001980FCF729
:10A8700033FF041E11D1002D0FD07689002E11D088
:10A880000C2001F099F800280ED0084A04601368E3
:10A8900086808560002B02D11060200076BD1A00F2
:10A8A0001B68F7E70224F8E71324F6E7A06BFF1F05
:10A8B000012100220A4B10B549420A4C19809980A7
:10A8C0009A719A70084B2070012019805A60FFF726
:10A8D000A3FF2078FCF75EFF0448FDF719FF10BDC9
:10A8E000A469FF1FA86CFF1FA06CFF1F9DA900118A
:10A8F000022310B5002802D0FFF7B2FF03001800B2
:10A9000010BD0000030010B50020DB0704D50421B2
:10A91000024A0348FFF7A4FF10BDC04628BE00113D
:10A920003845FF1FF0B50E2687B003930CAB1F8888
:10A9300002ABF6180500080031000292FDF74EF850
:10A9400004000120002C0FD03088FFF74BFF0300DC
:10A950000E20002B08D05E68002E05D021002800B4
:10A96000039B029A0097B04707B0F0BD0A4B10B5A1
:10A97000984207D10122002352420A808B708A80BC
:10A980008B7110BDFFF73CFF0028FAD001235B421A
:10A99000038000238370F4E7FFFF0000F8B5050093
:10A9A00001290AD1134E00243388F827AB4219D06D
:10A9B00028001149FFF7DAFF06E0022904D1013926
:10A9C000FDF724FF0028EDD0F8BD3B00634372681B
:10A9D000D018D35A002B09D03A00002101F04CF8CE
:10A9E0000134E4B2054B1B78A342EED801235B424D
:10A9F0003380DDE7A06CFF1FA469FF1F9C6CFF1F65
:10AA000010B5FFF7FDFE03000020834200D09878C8
:10AA100010BD0000F0B589B01C000EAB80CB0390D8
:10AA20001E8810AB1B78049202930B7A0D00DB0694
:10AA300016D42B780593022B24D00498FFF7D2FE6E
:10AA4000002812D003689C46002B0ED0029B2200E7
:10AA5000019329003B00644603980096A04705E057
:10AA60000498FFF7BFFE002802D10E2009B0F0BD08
:10AA70008368002BF9D00A22290003989847002800
:10AA8000D7D0F3E76B6858781A786B4B0002104305
:10AA90009842D2D8043B984210D2684B984242D098
:10AAA00015D8674BC0180128C7D80B20002EDDD160
:10AAB000EB681A7859683A80200028E0614BC0188A
:10AAC000032800D979E000F05FFD846A789E5E4B30
:10AAD0009842B2D10B20002EC8D101233B80EB68F5
:10AAE00031001B7823706889013080B2FCF776FF53
:10AAF0003A88031E0ED0017802328A183A804289C1
:10AB000062704289120AA27059680278E01C00F053
:10AB10007BFF06E004323A8031000422601C00F022
:10AB2000ABFF0020A2E70B20002E9FD1EB6807A906
:10AB30001E8804233B80330A300026706370FCF7C4
:10AB40004DFF051E28D004AB9A890E2304A95B187B
:10AB50003E49C668FCF7B6FF00280BD12B783C486D
:10AB60006A680599FBF76CFB002803D1012304AA4E
:10AB70005B42D3813278022A06D17168201D00F031
:10AB800043FF3B8802333B800E2304AA9B181B889B
:10AB9000A3701B0AE370C4E704ABDE81F4E70B206B
:10ABA000002E00D062E7E9680398FFF729FF02232F
:10ABB0003B802070000A6070B3E70B20002E00D0AD
:10ABC00054E70222EB681B883A8023701B0A6370EB
:10ABD000A7E7E86800F000FFC2B203000720B24216
:10ABE00000D243E70DD00299DBB27118994202DB23
:10ABF000921BD3B20293029BE9681A003B80891929
:10AC00005AE70023F6E70B20002E00D02EE707229C
:10AC1000EB683A801A7822705A7862705A88A2706B
:10AC20005A88120AE2701A792271DA886271DB8816
:10AC30001B0AA37175E7C046042900000228000022
:10AC400000D8FFFFFFD6FFFF03280000FFFF000032
:10AC500058BD0011F0B58DB06B4600200891202240
:10AC60009B5E83423DDAA64B187800F025FC071E58
:10AC700032D00378B02B2CD10079023816281FD897
:10AC800000F07AFE17001E001E001E0031001E009C
:10AC900096001E001D011E0052011E0073011E00C1
:10ACA000CD011E0050021E001E001E008E021E005E
:10ACB000E302944B94491B8878880B80FBF700F8DB
:10ACC0003800FCF781FF914B1B68002B01D0380046
:10ACD0009847380000F088FC8020089B0002434021
:10ACE00018000DB0F0BDF6220021874800F0C4FE28
:10ACF0000BAA3B7B7989388900923A000D32FCF728
:10AD000085FD0400804B1B78002C3FD146E0804B32
:10AD1000788805937F4B4100CB5A0BAE073BDBB2E3
:10AD200032880293002301937B4B2100069300930A
:10AD3000059BFFF76FFE744D002810D1069B3A8AE1
:10AD40001B889A420BD138000599123000F0D4FBD1
:10AD5000002804D02B7862899B00EB185A801623B8
:10AD600006A81B18328820007989FCF7ABFE2B78E7
:10AD700004009A00AA1851880029C3D00133DBB21D
:10AD80002B70002807D006A9C98A9180634A1288CF
:10AD90009A42BCD802E0012149429180002B04D0A4
:10ADA00059497888FAF7C0FF8AE73E890A2479E092
:10ADB00000253E89574B06937B88069A5B009B5A79
:10ADC000033B9D4202DB002DF0D05BE0162206A87B
:10ADD00012183B7B798900923A0030000D32FCF763
:10ADE00015FD0590002858D04689017A7888FCF72F
:10ADF000D7FC041E44D1464B78880793069B41003C
:10AE0000C95A454B0439C9B206AAD28A069302919F
:10AE1000019400930599079BFFF7FCFD041E2FD1B9
:10AE2000069B39491A88931C002D26D14B807988BE
:10AE3000384B4900CB5A5119033B8B4220DD059B0F
:10AE400031485B8941190B71A91C0135C9B2EDB2BA
:10AE5000059145191B0A2B71059B2D4904331818C0
:10AE600000F0D2FD2C4B059A1B88D318DDB22C4B79
:10AE70009E4205D00136B6B29CE749889942D6D0A9
:10AE8000002D0CD0204C2800618800F06DFD207052
:10AE900021007888FAF758FF12E7059CF0E7002CAC
:10AEA00000D183E77B78142B00D109E716493B7961
:10AEB0004E800B700C717888FAF7F8FE00E71624C4
:10AEC00006ABE41821003889FCF788FD011E00D18B
:10AED000B7E1788822880F4C45002C5B0A4D013C75
:10AEE000E4B2029400240F4B01940095FFF792FD09
:10AEF000041E00D014E129007888FAF735FFDFE658
:10AF0000A86CFF1F2444FF1FAC69FF1FA069FF1F2F
:10AF1000A66AFF1FDC65FF1F9C6BFF1F2244FF1FFB
:10AF2000FFFF0000AE69FF1F162406ABE4182100E6
:10AF30003889FCF753FD011E00D182E17888228810
:10AF4000AE4C45002C5BAE4D013CE4B202947C89D2
:10AF5000AC4B01940095FFF75DFD041E00D0DFE0CF
:10AF600029007888FAF70AFFAAE60025A44B1D807D
:10AF70003B00FE331B78A24A78880792AB4208D97F
:10AF80009E4B12880693069943005B5A013B9A42F6
:10AF900003DB0799FAF7FCFE92E616246B00FB1818
:10AFA000059306ABE418059B21001889FCF716FDF4
:10AFB000011E03D1059B01241E8973E77888924BFB
:10AFC0002288069C099343001B5B904E013BDBB239
:10AFD0000293002300960193099BFFF71BFD041EBB
:10AFE00002D0059B1E895DE77B88069A5B009B5A11
:10AFF000079A108832881218934202DC1B1A013B10
:10B0000033807F4C023032880999001900F0FCFC33
:10B010002388328801359B182380EDB2A8E70BAA5C
:10B020003B7B7989388900923A000D32FCF7EEFBC0
:10B0300000250590059B002B04D10A24002D00D18A
:10B040006EE060E0059B7888197AFCF7A9FB0100A7
:10B05000041E63D1694C6C4B788806940993069B57
:10B060004400E45A694B063CE4B20BAE32880793C5
:10B070000294019100930599099BFFF7CBFC041EF4
:10B080004CD1079B5E491B881A1D002D30D14A8088
:10B09000059B5B4C5A8963191A716B1C9BB2E318B0
:10B0A000120A1A71162306A832881B187989059886
:10B0B000FCF708FDFF21AA1C2E1D03350B0005908F
:10B0C00092B2B6B2ADB2002803D006ABDB8AD9B2D9
:10B0D0001B0AA218651911712B714C4D301D2A885D
:10B0E0004949201800F090FC2B88F618B5B2A1E76A
:10B0F0004988914207D17A8806995200525AEB1832
:10B10000053A9A42C4DC3E4C2800618800F01CFCE1
:10B11000207021007888FAF745FED1E5002DF2D1A4
:10B120003E89BFE6162606ABF61831003889FCF7D3
:10B1300055FC3D000400FF3500282DD0037A9B0606
:10B140000CD400227B893989788800923A000C322D
:10B15000FFF7E8FB041E10D03E8915E03088FFF7AA
:10B1600041FB00281AD08368002B17D0210012223F
:10B1700078889847041EE4D0EEE7AB78002B02D124
:10B180007888FAF71FFE0026AB78002B00D097E5F1
:10B19000002C00D194E585E60124DDE70E24DBE7F1
:10B1A000162506ABED1829003889FCF717FC041E9C
:10B1B00047D0037A9B0611D4154A7B88118899429F
:10B1C00003D01448814207D11380134BF8261D7811
:10B1D0000023D9B2A94221D30924A1E72888FFF787
:10B1E00001FB00282FD08368002B2CD021001222D5
:10B1F00078889847041EDFD092E7C046DC65FF1FC1
:10B20000AC69FF1FAE69FF1FA66AFF1F9C6BFF1F83
:10B21000A06CFF1FFFFF00009C6CFF1F3100594313
:10B22000546801336018615A0029D2D13C000834B7
:10B230002100F82200F0E8FB21007888FAF7CAFD27
:10B240003EE501246CE70E246AE71D4B1A887B88D3
:10B250009A4231D07888FAF7C7FD31E5F82305988E
:10B2600051684343CD18C95A00291FD03B7A012B9E
:10B270000BD16C88AB887888AA1D0094FFF752FB2D
:10B28000041E02D000233B722E88F82200212800E1
:10B2900000F0F2FB00232B80059B0133DBB205930A
:10B2A000084B05991B78064A8B42D7D801235B428D
:10B2B0001380002CCED0F5E5002634000596EFE78C
:10B2C000A06CFF1F9C6CFF1F70B504000E001500E2
:10B2D000FFF796FA031E08D131000548FFF790FAF0
:10B2E00003001120002B02D01C8000209D7070BD37
:10B2F000FFFF0000F8B50B4F06003B780D0014006F
:10B30000FF2B0ED00A2000F0D7FB011E09D0B1237D
:10B310000380002346800371C5800481387800F0E3
:10B3200053FBF8BD7945FF1FF7B50F0008A90600CC
:10B33000088809A90B240988002821D10234022B8E
:10B340001ED1557813782D021D432B008B4301939A
:10B350007334002B14D1FB68300019000093FFF701
:10B360004FFB019C85420BD02A0030000099FFF76B
:10B37000ABFF041E04D12A0030007989FFF7BAFF21
:10B380002000FEBDF0B50E7885B003900AA80588B0
:10B390000120022E0DD14C682778647824023C43AA
:10B3A000054FBC4205D10398DBB201960095FFF72B
:10B3B000BBFF05B0F0BDC0460229000010B5040077
:10B3C0000C4800F019FB0C48A16B00F015FB0B4872
:10B3D000E16B00F011FB0A48216C00F00DFB094BFA
:10B3E0000948196800F008FB084B1B68002B00D0C7
:10B3F0009847FEE70EBC001124BC001133BC0011BD
:10B4000042BC001104ED00E051BC0011AC6CFF1F08
:10B41000002307B501A80193FFF7D0FF044A0548B0
:10B42000002110B5121A00F027FBF8F7C5FAFEE765
:10B43000B06CFF1F7C45FF1F01B40248844601BC6D
:10B44000604700BF353BFF1F01B40248844601BC82
:10B45000604700BF151BFF1F01B40248844601BCB2
:10B46000604700BFF94C010001B40248844601BCAA
:10B47000604700BF350E000001B40248844601BC9D
:10B48000604700BF8D12000001B40248844601BC31
:10B49000604700BF055E000001B40248844601BC5D
:10B4A000604700BFB54C010001B40248844601BCAE
:10B4B000604700BF6571010001B40248844601BCC9
:10B4C000604700BFF54E010001B40248844601BC4C
:10B4D000604700BF7D18FF1F01B40248844601BCCD
:10B4E000604700BFD1A5000001B40248844601BCFA
:10B4F000604700BF9DA9000001B40248844601BC1A
:10B50000604700BFCD4C010001B40248844601BC35
:10B51000604700BFA946010001B40248844601BC4F
:10B52000604700BFE139FF1F01B40248844601BCF7
:10B53000604700BFC9A9000001B40248844601BCAD
:10B54000604700BF0124000001B40248844601BCEA
:10B55000604700BFF30E000001B40248844601BCFE
:10B56000604700BF311B000001B40248844601BCA3
:10B57000604700BF017F000001B40248844601BC5F
:10B58000604700BFD91B000001B40248844601BCDB
:10B59000604700BF453CFF1F01B40248844601BC20
:10B5A000604700BFC94A010001B40248844601BC9B
:10B5B000604700BF851F000001B40248844601BCFB
:10B5C000604700BF213AFF1F01B40248844601BC16
:10B5D000604700BFC926000001B40248844601BC90
:10B5E000604700BFED4A010001B40248844601BC37
:10B5F000604700BF434D010001B40248844601BCCE
:10B60000604700BF014C010001B40248844601BC00
:10B61000604700BF6939FF1F01B40248844601BC7E
:10B62000604700BFC521000001B40248844601BC48
:10B63000604700BFC95C010001B40248844601BCF8
:10B64000604700BFC53F000001B40248844601BC0A
:10B65000604700BF2526000001B40248844601BCB3
:10B66000604700BF4134FF1F01B40248844601BC5B
:10B67000604700BFDD30FF1F01B40248844601BCB3
:10B68000604700BF2124000001B40248844601BC89
:10B69000604700BFB352010001B40248844601BCB8
:10B6A000604700BF691F000001B40248844601BC26
:10B6B000604700BF3D18000001B40248844601BC49
:10B6C000604700BF3555000001B40248844601BC04
:10B6D000604700BF5539FF1F01B40248844601BCD2
:10B6E000604700BF0D52010001B40248844601BC0E
:10B6F000604700BF5125000001B40248844601BCE8
:10B70000604700BF4D1F000001B40248844601BCE1
:10B71000604700BF75A9000001B40248844601BC1F
:10B72000604700BFA54F010001B40248844601BC38
:10B73000604700BF9938FF1F01B40248844601BC2E
:10B74000604700BFE548000001B40248844601BCE0
:10B75000604700BF093BFF1F01B40248844601BC9B
:10B76000604700BFB14E000001B40248844601BCEE
:10B77000604700BF5D17000001B40248844601BC69
:10B78000604700BF291C000001B40248844601BC88
:10B79000604700BFE928000001B40248844601BCAC
:10B7A000604700BFE117000001B40248844601BCB5
:10B7B000604700BF056A000001B40248844601BC2E
:10B7C000604700BFA139FF1F01B40248844601BC95
:10B7D000604700BF5118FF1F01B40248844601BCF6
:10B7E000604700BF4551010001B40248844601BCD6
:10B7F000604700BF5549010001B40248844601BCBE
:10B80000604700BF091B000001B40248844601BC28
:10B81000604700BF313CFF1F01B40248844601BCB1
:10B82000604700BF8132FF1F01B40248844601BC5B
:10B83000604700BF8D3AFF1F01B40248844601BC37
:10B84000604700BF810E000001B40248844601BC7D
:10B85000604700BF1147010001B40248844601BCA3
:10B86000604700BF5147010001B40248844601BC53
:10B87000604700BFB70E000001B40248844601BC17
:10B88000604700BF6DBC000001B40248844601BCA3
:10B89000604700BF7918000001B40248844601BC2B
:10B8A000604700BFC56D010001B40248844601BC79
:10B8B000604700BFF136FF1F01B40248844601BC57
:10B8C000604700BFC51D000001B40248844601BCAA
:10B8D000604700BF9130FF1F01B40248844601BC9D
:10B8E000604700BF8B52010001B40248844601BC8E
:10B8F000604700BF0933FF1F01B40248844601BC02
:10B90000604700BF2951010001B40248844601BCD0
:10B91000604700BFC132FF1F01B40248844601BC2A
:10B92000604700BF456B010001B40248844601BC7A
:10B93000604700BF6932FF1F01B40248844601BC62
:10B94000604700BF5522000001B40248844601BC94
:10B95000604700BF090E000001B40248844601BCE4
:10B96000604700BF9135FF1F01B40248844601BC07
:10B97000604700BF350E000001B40248844601BC98
:10B98000604700BF593CFF1F01B40248844601BC18
:10B99000604700BF8552010001B40248844601BCE3
:10B9A000604700BF0189000001B40248844601BC21
:10B9B000604700BF5952010001B40248844601BCEF
:10B9C000604700BF3D4B010001B40248844601BC02
:10B9D000604700BF594F010001B40248844601BCD2
:10B9E000604700BFDD52010001B40248844601BC3B
:10B9F000604700BFEDA5000001B40248844601BCC9
:10BA0000604700BFE53A010001B40248844601BC2A
:10BA1000604700BFE94C010001B40248844601BC04
:10BA2000604700BF4550000001B40248844601BC95
:10BA3000604700BF2146010001B40248844601BCB2
:10BA4000604700BF1D4B010001B40248844601BCA1
:10BA5000604700BFD949010001B40248844601BCD7
:10BA6000604700BFE537FF1F01B40248844601BCB0
:10BA7000604700BF090E000001B40248844601BCC3
:10BA8000604700BF154D010001B40248844601BC67
:10BA9000604700BF1537FF1F01B40248844601BC50
:10BAA000604700BFADAE000001B40248844601BC4F
:10BAB000604700BF0134FF1F01B40248844601BC47
:10BAC000604700BF1D4D010001B40248844601BC1F
:08BAD000604700BFA134FF1F15
:10BAD800000201030202030304030502060207022F
:10BAE800080209030A030B030C020D020E030F03DD
:10BAF800100311031303140315001600793D0011F8
:10BB0800AD3D001100000000020000001ABB00114A
:10BB1800192A0F180A000000F1590000FD2400003E
:10BB280041460100197E00112D9E001181720011FD
:10BB38001D7C0011B551001155AC0011614E00116A
:10BB4800713F0011A140001100000000161600000E
:10BB58000200000064BB0011F4FFF3FFD2FC0000F8
:10BB68008541001100000000000000005475796153
:10BB78000056302E370030303031006769746875F0
:10BB8800622E636F6D2F70767678005448303500DA
:10BB980002000000ACBB0011292A282A272A262ADD
:10BBA800252A242A0A180000E20400007102000075
:10BBB80078EC0000744000001027000060F00000DE
:10BBC80006640000204E0000000000000000000095
:10BBD8001F501D00023C0200000115000700000074
:10BBE800A302000030313233343536373839414218
:10BBF80043444546005048592B36325858504C5506
:10BC08005330353034005B48617264206661756C6E
:10BC1800742068616E646C65725D0A004C52202065
:10BC2800203D203078253038780A005043202020E5
:10BC38003D203078253038780A0050535220203D76
:10BC4800203078253038780A0049435352203D2067
:10BC58003078253038780A00C5550011195600117A
:10BC6800000000000200000078BC00116F2A6E2A54
:10BC78001A18D880F060FFFFFFFFFFFFFFFFFFF3F8
:10BC880003B59747D6F613F7D777E6F0A7F474000D
:10BC9800000001A0000000006410B71DC8206E3B22
:10BCA800AC30D9269041DC76F4516B6B5861B24DBB
:10BCB8003C7105502083B8ED44930FF0E8A3D6D625
:10BCC8008CB361CBB0C2649BD4D2D38678E20AA08D
:10BCD8001CF2BDBDFB349B5F80000080001000009B
:10BCE80000000000835E00110D750011A75E0011B1
:10BCF800157900112B5F0011EB780011A15F00117D
:10BD0800C1780011F35F0011897A00115B6000119E
:10BD1800897A00118D600011437A0011A15F00112A
:10BD28007978001119600011217A001100000000D3
:10BD380000000000FF600011217A0011616100110C
:10BD480025750011052A042A012A002A0229032838
:10BD58000128002801180018000000000000000059
:10BD68000000000000000087010102010201010239
:10BD7800010203030401030101010101030302019C
:10BD880003000D000E00100011001300140107013C
:10BD980008010A010B011C011D0204020502070229
:10BDA800080219021A021C021D03010302031700EC
:10BDB8000201000504000807000B0A001716001D01
:10BDC8001C010201010504010E0D011110011413DB
:10BDD800011716011A19020201020B0A020E0D02BE
:10BDE8001110021413021716030504030807030BA6
:10BDF8000A030E0D0001020307090A0B0E0F1011AA
:10BE080012141718191A1B1F202122009DA50011B2
:10BE180059A6001100000000020000005EBD0011DC
:10BE28000000000085B300110000000002000000BF
:04BE38005CBD0011DC
:020000041FFFDC
:1000000000000000D53E001120BB00111CBB0011F8
:100010008862FF1F000000000000000000000000D8
:1000200000000000000000000000000000000000D0
:1000300000000000000000000000000000000000C0
:1000400000000000000000000000000000000000B0
:1000500000000000000000000000000000000000A0
:100060000000000000000000000000000000000090
:100070000000000000000000000000000000000080
:100080000000000000000000000000000000000070
:100090000000000000000000000000000000000060
:1000A0000000000000000000000000000000000050
:1000B0000000000000000000000000000000000040
:1000C0000000000000000000000000000000000030
:1000D0000000000000000000000000000000000020
:1000E0000000000000000000000000000000000010
:1000F0000000000000000000000000000000000000
:1001000000000000000000000000000000000000EF
:1001100000000000000000000000000000000000DF
:1001200000000000000000000000000000000000CF
:1001300000000000000000000000000000000000BF
:1001400000000000000000000000000000000000AF
:10015000000000000000000000000000000000009F
:10016000000000000000000000000000000000008F
:10017000000000000000000000000000000000007F
:10018000000000000000000000000000000000006F
:100190006534FF1F5533FF1FC166010000000000DA
:1001A000000000000000000000000000000000004F
:1001B000000000000000000000000000000000003F
:1001C000000000000000000000000000000000002F
:1001D000000000000000000000000000000000001F
:1001E000000000000000000000000000000000000F
:1001F00000000000000000000000000000000000FF
:1002000000000000000000000000000000000000EE
:1002100000000000000000000000000000000000DE
:1002200000000000000000000000000000000000CE
:1002300000000000000000000000000000000000BE
:1002400000000000000000000000000000000000AE
:10025000000000000000000000000000000000009E
:10026000000000000000000000000000000000008E
:10027000000000000000000000000000000000007E
:10028000000000000000000000000000000000006E
:10029000000000000000000000000000000000005E
:1002A000000000000000000000000000000000004E
:1002B000000000000000000000000000000000003E
:1002C000000000000000000000000000000000002E
:1002D000000000000000000000000000000000001E
:1002E000000000000000000000000000000000000E
:1002F00000000000000000000000000000000000FE
:1003000000000000000000000000000000000000ED
:1003100000000000000000000000000000000000DD
:1003200000000000000000000000000000000000CD
:1003300000000000000000000000000000000000BD
:1003400000000000000000000000000000000000AD
:10035000000000000000000000000000000000009D
:10036000000000000000000000000000000000008D
:1003700011B40011000000000000000000000000A7
:10038000000000000000000000000000000000006D
:10039000000000000000000000000000000000005D
:1003A000000000000000000000000000951AFF1F80
:1003B000000000000000000000000000000000003D
:1003C000000000000000000000000000000000002D
:1003D000000000000000000000000000000000001D
:1003E000000000000000000000000000000000000D
:1003F00000000000000000000000000000000000FD
:08183800B070FF1F4118FF1FF3
:10184000024981F3088802F04BFA0000B070FF1FD4
:1018500010B502F0BDFA072804D0122808D00228DB
:1018600008D010BD044A0420136B01331363F8E75A
:101870000220F6E71420F4E78466FF1FF8B507009E
:101880000C0026002500503630785135002804D150
:101890000300287058342370F8BD2978CA00481E08
:1018A0008141A3183800A25C5B68C9B2FFF7D0FF82
:1018B00000280DD12B78DA00A218013350602B706C
:1018C0003378044A013B3370136A01331362D8E75B
:1018D0000123DFE78466FF1F5C234343074910B5FC
:1018E000C9180B0058331B78012B05D1FFF7C6FF31
:1018F000034A936A0133936210BDC046B866FF1F66
:101900008466FF1F10B502F09BFA064A01211300FE
:1019100010CB4942D967044B136002F0F9FB200059
:1019200010BDC04600E100E01000100010B504003A
:1019300002F086FA024B1C6002F0EAFB10BDC046C2
:1019400000E100E010B5040002F07AFA4021094AF3
:10195000200013688B43136002F0FAF901F064FD74
:101960000022054B01201A60044B04321A6002F079
:10197000AFFBFEE71CF00040C4F00040C0F00040A8
:10198000431E5A425341A022F0B5D2015B4213409C
:10199000154D164A40019B182A18127E8BB00191F2
:1019A000002A1BD01A000832D46F0022E6B206AF1C
:1019B000E4B294420EDC2818C369002B08D00199C8
:1019C00002AA117106AA049202AA167303A89847E4
:1019D0000BB0F0BD1978B9540132EAE71A7D1A78D4
:1019E00006AB01261A70E6E74469FF1F004000407D
:1019F000F0B5254B04004001C25C85B0002A2BD015
:101A00001A18117E002927D0917E002924D011793F
:101A1000022921D11689D788D168F51BADB22A1CBD
:101A2000102D00D9102292B2BE4217D118180123EE
:101A300003710023C269C38003819A4206D06846BD
:101A4000032103730171029301A890470820002C21
:101A500000D0192001F034FC05B0F0BD013C654216
:101A60006C41A0256442ED012C40084D1B186419FF
:101A7000074D0633013A92B2AA42EDD01888461CAF
:101A80001E80085C2070F5E74469FF1F004000409D
:101A9000FFFF00000F220E4B10B59868104002386F
:101AA0000A280BD802F0CEF80D0A0B0A0A110A0A0E
:101AB0000A0A060002210020FFF762FF10BD012183
:101AC000F9E70020FFF794FFF8E7DB6FF6E7C04681
:101AD000004000400F220E4B10B5986810400238AD
:101AE0000A280BD802F0AEF80E0A0B0A0A120A0AEC
:101AF0000A0A060002210120FFF742FF10BD012162
:101B00000800F9E70120FFF773FFF7E7DB6FF5E760
:101B10000090004013B5334C2378072B3DD8324B4F
:101B20001A78324B002A39D18022196852020A43AE
:101B30001A60252001F034FF20232D4A11680B4341
:101B4000802113606B460422C905086807331042E0
:101B500028D080210422C905C86810422ED08021D7
:101B60002020C905CA688243CA6014221A701A78F4
:101B7000002A2FD18021C905C86820320243CA60DB
:101B800014221A701A78002A28D11A4B1A7D22784A
:101B90005A601D221A705932DA6013BD1A6816494C
:101BA0000A40C5E7086802430A6014221A701A78CE
:101BB000002ACED01A78013AD2B2F7E7C8680243B9
:101BC000CA6014221A7019784A1ED2B21A700029FB
:101BD000F9D1C4E71A78013AD2B2C7E71A78013AC4
:101BE000D2B2CEE7B444FF1F7C45FF1F3CF000405B
:101BF000AC44FF1F00200040FFFFFEFF564B70B5B6
:101C00001B68012B03D1554A936D0133936502F094
:101C100067F9534B534A1860534B544C1A600123D5
:101C2000534A1360534A13602378002B06D00622D0
:101C30005149524802F0A4FA00232370504A514BF4
:101C400010681B78C1B2002B0ED14F4CC0B2237864
:101C50005BB2002B4FDB237824785BB264B21B04A9
:101C600024021B191B1813600B1C50294ED950233A
:101C7000464A47491078DBB2FF2202284BD1086858
:101C8000444C454D267890432A78964254D9227880
:101C900024782E78023B5D10A31B6B435201D31AAC
:101CA00010335B111843086002F0E2F9031F012BA7
:101CB00045D83A4B1B78002B06D0394B1B78002BAC
:101CC00002D0002002F02CFAA122364B9200997823
:101CD000354B4A431B689B18832292009B181B7844
:101CE000033B012B03D8AF20400001F0E9FF0122A4
:101CF0002E4BDA8270BD237824785BB264B2FF3356
:101D0000FF341B0424021B190138ABE7CAB2022AB4
:101D1000AED20223ACE70868254C264D26789043C6
:101D20002A78964208D9227824782D78023B5B10D5
:101D3000641B63435201B2E72378DBB2B2E70228A7
:101D4000D5D11D4B1B78013B022B03D91B4B1B78B4
:101D5000022BCCD16C20C8E79809FF1FFC0FFF1F96
:101D6000BC65FF1FFF3F000014100340C065FF1F4C
:101D70000C10034000100340D50BFF1F7211FF1F12
:101D8000B40003408C09FF1F680AFF1F490AFF1FA8
:101D900094000340460AFF1F470AFF1FF908FF1F70
:101DA0002209FF1F300DFF1F3409FF1FBC0BFF1F4F
:101DB000440AFF1F450AFF1F1C09FF1F2309FF1FBD
:101DC00010B501F0FDFF0022014B1A8010BDC04686
:101DD000B865FF1F10B502F063F8A121054A89001C
:101DE0009478054A61431268044B5218528C1A8049
:101DF00010BDC046300DFF1F3409FF1FB865FF1F1F
:101E000010B50D4B0D4A9978A1239B004B431268E6
:101E1000D218531DD97F0A4B1B88994209D2441C02
:101E200007D0C82805D0D2695B1A5A43054B5343E3
:101E3000C01801F03DFF10BD300DFF1F3409FF1F1A
:101E4000B865FF1F7102000070B5244D2B68002B90
:101E500028D002F065F82B68D8402B680400002BCE
:101E600027D001F0CDFF2B68D8401D4B1D4A997833
:101E7000A1239B004B431268D118D25C91239B0095
:101E8000002A20D0CA580132CA50174B17491B6884
:101E90000868834214D3D23B181A012A1AD0144B73
:101EA000186070BD02F03CF8124B196801F010FF89
:101EB000D3E701F0A5FF0F4B196801F009FFD4E744
:101EC0000D495B18E8E7CA500C4B1B68DB68E41847
:101ED000201AE4E7F530FF30E1E7C0461C08FF1F99
:101EE000300DFF1F3409FF1F9C09FF1FBC65FF1F3A
:101EF000A009FF1F1808FF1F2DFF3F00C465FF1F2B
:101F000070B504000D00282916D10300A433C2883F
:101F10001B889B1A0B4A9BB293420DD906006A3666
:101F200005223100653002F023F9002804D1310088
:101F3000200001F0A5FF70BD2900200001F0C8FFBE
:101F4000F9E7C046FE7F0000F8B50400012002F06A
:101F50001FF801F0D5FF174A174910600968030000
:101F60001648174E01601748776805680020AF4291
:101F700001D27068281A144D091928601348C162EB
:101F8000A421446A49032143416211490978002987
:101F900005D010490978022902D10F3B1360F8BD22
:101FA000012901D1083BF9E7032901D1053BF5E7F8
:101FB000033BF3E7E408FF1F28F00040340AFF1F4B
:101FC00028100040180AFF1F1C0AFF1F00F00040E5
:101FD0001C09FF1F4A0AFF1F70B580241025E40565
:101FE000A3682B43A36001F053FFA368AB43A36036
:101FF00070BD0000F7B5160080221C001023D2052A
:102000000191916805000B43936000225A4BD73031
:102010001A6002F0BDF89D232A002F009B00EB58A8
:10202000CA3201210092FC37002B01D00021009A16
:10203000386801F0A5FF2900009BCB311A784F4B7F
:10204000D3351A604B780A781B0213438A7812043E
:102050001A43CB781B061343494A1BBA13604B79CA
:102060000A791B0213438A7912041A43CB7931008F
:102070001B061343434A1BBA13606B782A781B0272
:102080001343AA7812041A43EB781B0613433E4A03
:102090001BBA1360019A330213433C4A13603C4B52
:1020A00022001B1B9C4603293DDCB3089A00130049
:1020B0005142B21A032A46D1354AE018511A8278A1
:1020C0004078120400020243E05C043302430A60D9
:1020D0000022FF2B4BDDF0222E4B12011A600F2243
:1020E0002D4B1A602D4A1368002BFCD00023224A86
:1020F00027491360091B321D0B191B68043A180A83
:1021000023706070180C1B0EA070E3700434002A5A
:10211000F2DC802210213B68D20501333B609368DA
:102120008B439360F7BD6346D578981893782D0656
:102130001B042B43157804392B43557804322D02A8
:102140002B430360AFE7022A0AD1114AE05C511A1F
:10215000E2185278120202430A6004339BB2B7E7D6
:10216000012AB5D10A4A521AE15C1160F5E7084923
:1021700059180A600433ACE7000004403C000440F6
:102180003800044034000440300004400C00044097
:102190000001044004000440100004401400044006
:1021A000F7B5150080221C001023D205009191681C
:1021B00007000B4393600023654AD730136001F09A
:1021C000E7FF9D233E009B00F9583B00CA363200D2
:1021D000FC33002900D07FE0586801F0D1FE3900BF
:1021E00032785C4BCB311A604B780A781B02134370
:1021F0008A78AC4612041A43CB78281D1B06134379
:10220000554A1BBA13604B790A791B0213438A792A
:1022100012041A43CB791B061343504A1BBA1360AE
:102220004B7A0A7A1B0213438A7A12041A43CB7A36
:1022300021001B0613434A4A1BBA1360009A2B0263
:102240001343484A13602200474B1B1B0093009B1B
:10225000CE785B1801938B7836061B0433430E78D7
:10226000043833434E78043136023343019E3360E1
:102270000328ECDC0321A808431C9B0029408000B4
:1022800003292BD13849E5185E18A9786D78E35CED
:1022900009042D022943194331600300083300214A
:1022A000FF2B2DDD314B324919600F21314B196065
:1022B000012327490B60304B19680029FCD0062107
:1022C0001B680B40042B20D080220020D20593688D
:1022D0000A318B439360FEBD01217DE7022908D1BD
:1022E00021495D18E1184978E35C09021943296026
:1022F000D3E70129D3D11C495918E35C0B60CCE723
:102300001948181801600433CAE7002310490B600C
:102310006346002B0CDC3B00FC335A681021013271
:102320005A608022D205936801208B439360D2E7E4
:10233000009B9B181B68190A13705170190C1B0E17
:10234000D37004235B4291709C440432E0E7C046A2
:10235000000004403C0004403800044034000440C5
:10236000300004400C00044000010440040004401C
:10237000080F0000100004401400044070B5061E51
:1023800019D00222614B9B799343012B13D1604BEF
:102390001A78FF2A0FD15A78FF2A0CD19A78FF2A8F
:1023A00009D1DA78FF2A06D11A79FF2A03D15B799D
:1023B000FF2B00D1A7E0574B0C201A78012A08D038
:1023C0000022554D1A702B781A00093A042A01D8B8
:1023D000212070BD5A1F012AFAD94C4CA07B042839
:1023E00000D990E0A279032A00D98CE0821E012A4C
:1023F00003D862881F2A00D885E0002E61D0012E04
:1024000000D080E0A288012AE2D0002B0AD1013856
:10241000032803D801F016FC151D19151F202E7076
:1024200001F0BEFD2B785A1E032A16D800253B4B1F
:102430001D602823237501F0F3FCA8422ED0A5804F
:10244000C6E7022320202B70EAE7042322202B700A
:10245000E6E7032321202B70E2E7073B012BB7D8E7
:102460002F4B1B68DB6A9B06B2D52E4B1A78002ACD
:10247000AED1A27B911E012901D9002AA8D1022246
:1024800080211A702823284D89012878237501F0AE
:10249000BFFD80212878890101F06AFD0123A38016
:1024A000224B1B78002B0AD0FA228021204B92006D
:1024B0001B8809025A431C4B187801F071FE00205A
:1024C00087E701F0BDFC2B78A680073B012B06D9DE
:1024D00018482E7001F08CFC1E2001F061FD114B9C
:1024E000114C1A78002A06D0802100222078890118
:1024F0001A7001F08DFD01F00BFE80212078090299
:1025000001F086FDDBE7122063E7C046A60BFF1F44
:102510006B09FF1F1A09FF1F1C09FF1F4809FF1F36
:10252000C465FF1F2309FF1F1B09FF1F2109FF1F90
:102530002C09FF1F0010004010B5002901D001F048
:10254000F7FD10BDF7B5604B01919978A1239B0071
:102550004B435E4A060014681022E418D6235B0041
:10256000E0583623FF33E35C00279343222B41D10D
:10257000574B0F3A1A600760012501F011FC019BCF
:102580001880E8235B00E35C002B01D0B34258DDE8
:102590000023504FFB70AD33FF33E3581A68002A15
:1025A00003D09B88DB439B071DD03823FF33E35CBC
:1025B000002B18D09B235B00E35C002B13D1D1339D
:1025C000FF33E35CB3420EDAA4235B00E15AE01868
:1025D000090A023101F044FC23000122FE33013ECE
:1025E00001351A87FA70E8235B00E35C002B2AD0E0
:1025F000A8B2FEBD03683D00002BBED08188043028
:10260000090A023101F02CFCD6235B00E3581F605D
:10261000B2E72300B133BA00FF33985801378188FD
:102620000430090A023101F01BFCE8235B00E35C83
:10263000BB42EEDCE822F61AED1800235200A35448
:10264000A6E70027F1E7200001F02AFB00281FD0B1
:10265000002E1DDD7319882647190193B60020004E
:1026600001F086FB5A3080002018406801358188CF
:102670000430090A023101F0F3FB200001F070FD83
:10268000A3590133A351BD4202D0019B9D42E6D123
:10269000114BE35C002BABD095239B00E35C002B3C
:1026A000A6D00E4BE15A0029A2D00D4AA35C994254
:1026B00002D90133A3549BE700231A212000A3541D
:1026C00001F0BEFC94E7C046300DFF1F3409FF1F28
:1026D00000140340E010FF1F5A02000072020000C5
:1026E0005E020000F8B51D4B1D4F1A78002A10D16C
:1026F000BA7B002A02D101321A7003E0032AFAD011
:10270000022AF8D001F08CFB00220120154B1A7030
:10271000F8BD154B154D1C68154B9E7801232B7089
:102720002878C0B200F0DEFCBB7B002B0BD101F09F
:10273000E7FCA1239B007343E41883239B00E41868
:1027400023782B70E4E7032B02D101F059FCF0E76A
:102750000020022BDCD101F0B3FCEAE71C09FF1FCB
:10276000A60BFF1F2309FF1F3409FF1F490AFF1F84
:10277000300DFF1FF0B587B00EAD2F780FAD2D785F
:102780000593AC46634614000E4D0CAA12782E78C1
:1027900003930D9B009201932200059B029701F089
:1027A000D7FC2E70012C01D0042C08D180220649C0
:1027B0008B889343054A1278D20113438B8007B06C
:1027C000F0BDC0461C09FF1F6C11FF1F7809FF1FD9
:1027D0000B001B3B70B504003020E02B0DD813001C
:1027E000E025493BFF3B9BB2ED00AB4205D8034BD4
:1027F000200019825A8201F0DBFB70BD8410FF1F9C
:1028000010B501F06DFB054B00205B68052B04D96A
:10281000034A5268D20200D4980810BD001000404C
:10282000FCE100E070B501F00BFB0D4B1B68FC33C5
:10283000DC691D6AFFF7E4FF6419844204D2094B86
:1028400001241B68002B07D004220024064B1A70B9
:10285000064A93690133936101F05AFC200070BD70
:10286000C465FF1F9809FF1F2309FF1FFC0FFF1FEF
:1028700070B50C4D2B68FC335C6A01F0E1FAFFF790
:10288000BFFF2B680025FC339B6AE318834204D208
:10289000054B1B68AB4200D1051B01F039FC280039
:1028A00070BDC046C465FF1F9809FF1FD722044BA7
:1028B00092009B5810B5002B00D0984710BDC04621
:1028C0000000FF1FF0B587B001F046F9FFF7EEFFFB
:1028D000CA4BCB4C04931B78022B45D1C94B1B68C8
:1028E000186A01F055FBC84BC84A1A60C84BC94A60
:1028F0001A60A022C84B52001A60049B187801F09D
:102900006FFBC649C64801F0BBF9C649C64801F08D
:10291000B7F91022C54BFF201A60802252031A60BB
:10292000802292031A60802212041A6001F0F8FBE0
:10293000012001F03DFAFA20400001F0A1FB5820EF
:1029400001F0BEF9BA4801F063FA012001F038FB4A
:10295000072001F0F5FA2268B64B1A4084235B0089
:102960001343236007B0F0BD01F09AFBB24E029012
:10297000322001F00DFB33681B0629D43C2001F006
:1029800007FB0F2001F004FB9C4B1B78012B00D1AF
:102990001EE180223368A94D134200D0A7E02B68C6
:1029A000032013432B6001F0F3FA01F079FB029B43
:1029B0000299C31A5A1E814200D81A00A04B1A600D
:1029C000904B19681E2353439E4A9B18CB618AE79C
:1029D00001F066FB80239C4ADB02116803900B43E5
:1029E00013602268934B994F1A40282313432360A6
:1029F000032001F0CDFA03203D6801F0C9FA3B68DD
:102A00000320DB03DB0B009301F0C2FA3B68ED030C
:102A1000DB03ED0BDB0B8E4A0193AB18C22B30D8D6
:102A2000009B9B18C22B2CD8019B9B18C22B28D82B
:102A3000009B2A009D4200D21A00009B9D4200D9B3
:102A40001D00019B934200D21300019A954200D9C8
:102A500015005B1B122B14D80C22336814209343EF
:102A6000336033687B4A1340336001F091FA0821E8
:102A70003B682268DB038A432260774ADB0B1360E2
:102A80007FE7032001F084FA3B68DB03DB0B05934F
:102A900001F006FB039B0399C21A531E814200D822
:102AA00013006E4A93421BD9FF23356869492D0AEA
:102AB0001D4032686B1C1B060A401B0C134333601D
:102AC0000C23326800209A43083B1343336001F023
:102AD00087F96348634BA840984206DCFEF732FF53
:102AE000019B009D0093059B95E75F48F6E7002357
:102AF0005E4F554A3B6080231168DB020B43136035
:102B000080222B68032013432B6001F041FA3B68BD
:102B1000052601333B6080232A685B0213432B6048
:102B20002268444B03201A40514B1343236001F0A9
:102B30002FFA0821454B1A682368D2038B43236080
:102B4000454B023900931B68D20B4B439A420CD879
:102B50009B1A3B2B0BD8236846490B4023602B68FC
:102B60000B402B60444B1A601FE7D31AF1E7013E7C
:102B7000F6B2002ED4D123683E4A134023602B685E
:102B800013402B603B68042B07D9BFF34F8F3B4B9F
:102B90003B4ADA60BFF34F8FFEE780222B680320A9
:102BA00093432B6001F0F4F92268224B03201A4072
:102BB00028231343236001F0EBF9244B009A1B6890
:102BC000DB03DB0B1360082223689343236097E742
:102BD00007222C4D2B681340012B02D1002001F05D
:102BE000FFF9AB68284A02201340AB6001F0D0F92E
:102BF0008023AA685B001343AB60D6E64A0AFF1F36
:102C00005CF00040C465FF1F000003400180063DEA
:102C1000BC00034034080000A4000340710200001F
:102C200014100040FFFF3F002810004000E100E0CA
:102C30003075000000FEFEFFC4F0004044F000408C
:102C4000AC65FF1F7206000040F0004064F00040D9
:102C500091FCFFFFFF00FFFFB465FF1FE30C0000C6
:102C6000E88000005F361E0060361E001844FF1F1B
:102C700028000100FFFFFEFFB065FF1F00ED00E030
:102C80000400FA053CF00040FFFEFFFF694E336888
:102C900088331B6883F3088801F02AF900F0C4FB2D
:102CA000654B664A1B68934207D0002001F098F8F4
:102CB0000221634A13688B431360FFF703FE614BE5
:102CC000614C1878C0B201F0CBF90023A360023345
:102CD000A3605E4B0120236001F05AF90323A36037
:102CE00001F0DEF9040001F0FBF8050001F0D8F96D
:102CF000574B186001F0DCF9564B1968621A531EE5
:102D0000A14200D213008022D203934201D39B023E
:102D10009B0A3268D16AC90700D478E04E491C0C7E
:102D200009689BB24C4359432402090A64180327DB
:102D30004A49FC3293680A6849489B1A494A4A4EF4
:102D400012684A499B18414A34609A183B400193E3
:102D5000036892089C46019B0A6063440360042B4D
:102D600003D901323B400A6003600B684049E41814
:102D7000200000F0ADFF3F4F3D493B68C3183B606A
:102D80002000019300F0B4FF3B4C2068081838493C
:102D90002060884205D9019B01333B6000F0A8FF09
:102DA000216000F0EDFF354B1B78002B0ED001F0B9
:102DB00097F83168324B4A1B1B6812189A4233D27B
:102DC000591A4919091A2F4800F05AFF2E4C237A34
:102DD000002B0FD001F084F83168E3684A1B121809
:102DE000934224D9591A4919091A284800F048FF72
:102DF00000232372264B83F3088800F0C9FF0220CA
:102E000001F0CEF8002000F0EBFF01F009F9DC0141
:102E100099000234641A5900641A09214B43803323
:102E2000CB40A408E41882E7FA218900CBE71949CE
:102E3000DBE7C046C465FF1F0C0AFF1FB641210334
:102E400010000040490AFF1F14100040C409000090
:102E5000100AFF1F340AFF1F380AFF1F200AFF1F36
:102E6000280AFF1F1C0AFF1FA865FF1F240AFF1F57
:102E7000710200006008FF1F2C0AFF1F1C09FF1FC2
:102E8000E408FF1F00100040740BFF1F3C100040BF
:102E900000000020DC050000A022054B92009B589A
:102EA00010B5002B01D0984710BD01F0D1F8FBE719
:102EB0000000FF1FA122054B92009B5810B5002B6C
:102EC00001D0984710BD01F0C3F8FBE70000FF1FD9
:102ED000A222054B92009B5810B5002B01D09847B9
:102EE00010BD01F0B5F8FBE70000FF1FA322054B62
:102EF00092009B5810B5002B01D0984710BD01F0EF
:102F0000A7F8FBE70000FF1FA422054B92009B5887
:102F100010B5002B01D0984710BD01F099F8FBE7E0
:102F20000000FF1F70B500F0DBFF514B186004205C
:102F300001F036F800F004FF0400C30702D400F0EB
:102F40000FFF70BD00224B4B1A604B4B18780138B5
:102F500004282CD800F076FE03231B1F2700200036
:102F600000F0AEFF0128ECD0444C2378042B71D143
:102F700001F03EF8002806D000F08AFE582000F04C
:102F80009FFE02232370032001F00AF8D9E72000F6
:102F900000F0CEFFE6E7200000F0E2FFE2E72000CD
:102FA00000F066FEDEE7200001F042F8DAE701F00B
:102FB0005FF80500012808D1314B1B78053B012B38
:102FC00003D82000FFF768FFCEE72C4B1B78022BBD
:102FD00001D0052B20D1022D28D12A4B9B7BAB435E
:102FE0001CD12000FFF766FF254B18780128BBD1C4
:102FF0006405B9D4234925224B7B034205D1233AEA
:1030000013405A42534126331A000B7D9342ABD9E9
:10301000322001F03DF8A7E7022D07D1184B1B78AD
:10302000052B11D12000FFF753FFDDE7012D0BD158
:10303000012B03D12000FFF759FF95E7062B03D1A1
:103040002000FFF761FF8FE7200001F001F8022D5B
:103050008AD1C9E7032B04D10B4B987C01F048F8C7
:1030600091E7072B8FD1094B987B00F061FE8AE72F
:103070009C09FF1F9809FF1F9009FF1F2309FF1FCD
:103080001C09FF1FA60BFF1FBC0BFF1FD40BFF1F4C
:10309000FA210A4B0A4A49001A640A4A5A500A4A53
:1030A00004395A50094A08319A64094A5A50094A5F
:1030B0005C315A50084ADA667047C0460000FF1F6C
:1030C0007527FF1F7128FF1F2528FF1F7D23FF1F66
:1030D000E526FF1F011EFF1FD51DFF1F10B500F0C5
:1030E00099FD10BD8023F7B59C46264B264F0193D2
:1030F0002649274A274D284C284B02281AD16046DA
:1031000038600868264E3040802636033043086019
:1031100001990978002909D11660224A2A60224AB9
:103120002260E02219689143A03A1BE08021C90285
:103130001160F2E766463E600F68194E3E408027F8
:10314000FF023E430E600199097800290DD11760F6
:1031500001280ED1154A2A60154A2260E02219681A
:103160009143C03A0A431A60F7BD80218902116079
:10317000EEE7E0210F4A02432A600F4A22601A68F4
:103180008A43F0E74B0AFF1FE0000340D8000340EA
:103190009000034000000340500003404000034003
:1031A000FFFFE3FF0280063D804508220180063DC7
:1031B000806608220080069880550822F8B51E4BCC
:1031C00080261A68002014003440324232D11A6836
:1031D0001A4F32431A6001223B68063093433B602A
:1031E00000F0D6FE0122164D2B681E432E603B6870
:1031F0000A2613433B608027BF00124B1B683B42EB
:1032000011D1013EF6B2FF2E09D17E220E4B1C6871
:103210002B68E40B1440934323432B6005E0082004
:1032200000F0B6FEE9E7002EEFD180222B6860089F
:1032300093432B60F8BDC046C4F000405CF00040F2
:1032400018F0004068F0004060F0004010B500F059
:10325000EFFD01215820034A00F062FDFFF7AEFFA9
:1032600010BDC046600AFF1F10B578220021034838
:1032700000F04EFD00F0ECFD002010BDCC68FF1FFB
:1032800070B5040000F0DCFD00230C200B4A0100A7
:1032900059438D18515C00290DD0A14208D101235A
:1032A00000246B7000F04CFF00F032FF200070BD76
:1032B00001330A2BEBD11224F6E7C046CC68FF1F7E
:1032C00070B5040000F0BCFD002319001D000D4A7C
:1032D0001078002806D0A0420CD1557001310C3274
:1032E0000A29F5D1002B0AD100F0B2FD00F010FF41
:1032F000002070BD5078461EB0411B18EEE700F06C
:103300001FFFF3E7CC68FF1FF7B504000C20002374
:1033100084460E4D019267465F43E85D7E19A042E8
:1033200012D000280BD10A4B9C4662461B7808330A
:103330001370019B70707C557160B360FEBD0133EA
:103340000A2BE8D10320F9E70720F7E7CC68FF1F35
:10335000C868FF1F8021204BC9051B6870B58B60B2
:103360001E4BC1241A680123FF2013434B611C4BE1
:10337000A4001A681B4B00251A601B4B1A681B4BD4
:103380001A601B4B1A5982431A51C52292009C584D
:103390008443BF38204398509C58164804408020EE
:1033A000C001204398509858134C0002000A014372
:1033B0009950124B1B78DB08AB4201DC002070BD3A
:1033C0002378002B06D0A368002B00D09847013546
:1033D0000C34EEE71220F2E7B044FF1FAC44FF1FAD
:1033E000B0F00040C468FF1FB4F00040C068FF1F89
:1033F00000E100E0FF00FFFFCC68FF1FC868FF1F6F
:10340000030010B51F2809D8072200201340072405
:1034100004490A78A24313430B7010BD0023062011
:10342000F5E7C046C868FF1F034A04491368002037
:103430000B4013607047C0461CF00040FFFFC1FF07
:10344000054B06491B780A6805485B0702401B0BC1
:10345000134300200B607047C868FF1F1CF000403A
:10346000FFFFC1FF70B50C25FFF7EAFF0A4B1C7880
:103470000A4BE4086543ED18002C01D1200070BD13
:103480002B78002B06D06B68002B00D09847013CAE
:103490000C3DF1E71220F2E7C868FF1FC068FF1F6C
:1034A00007B50422074801A900F034F9019B013354
:1034B00005D18023044ADB0411680B43136000200C
:1034C0000EBDC0461C18001114F00040F0B50500F8
:1034D0002026184B87B00493049B002B03D11124A2
:1034E000200007B0F0BD002102220B0001910091E5
:1034F000052000F06DFD02230F490A681A42FCD135
:103500000596059C631E0593002CFAD10B4A13689F
:10351000002BFCDA0F276F440121380000F0A8FCD3
:103520003B782B42DCD0052000F032FD049B013BB0
:103530000493D1E7FFFFFF0790C8004000C8004098
:1035400007B500F07DFC80220821D205936A019125
:10355000002B01D10739916202210C4A11600199B7
:10356000481E01900029FAD1033111600531019103
:103570000199481E01900029FAD11160002B02D157
:103580008022D205936200F0C3FD07BD00C0004059
:10359000F0B52D4C89B02378002B4FD1FEF7B2F94E
:1035A00002232A4F03903A681A42FCD12023069343
:1035B000069B5A1E0692002BFAD1254E3368002B2B
:1035C000FCDA0120FFF782FF011E02D0112009B0B2
:1035D000F0BD030003220190009005AD9F2000F094
:1035E000F7FC0321280000F043FC02233A681A424A
:1035F000FCD120230793079B5A1E0792002BFAD178
:103600003368002BFCDA0120FFF760FF0028DDD1D2
:103610000398FEF78BF9AA786B7811041B020B4311
:1036200029780B4363601300113B0A49052B07D827
:1036300001239340A3600B60012323700020C6E7A1
:1036400080231B03F6E7C0469844FF1F90C8004044
:1036500000C800409808FF1F1E4B30B55A68187804
:103660001D4B85B0D31859424B41012100930023D3
:1036700000F09EFD194B1A4A02259A6300221A6532
:1036800010325A658022C4219D65164B1648D2021D
:10369000DA6789004258154B80241A4080231B04A6
:1036A00013434350642341200393E40500F078F969
:1036B000402000F075F96562039D6B1E0393002D99
:1036C000FAD103236362FFF73BFFA562FFF760FFB8
:1036D00005B030BDA444FF1F95FFFEF700C80040B1
:1036E000050001FF04E100E000E100E0FFFF00FF52
:1036F00010B5064B18705960FFF7AEFF002113207C
:10370000034AFFF701FE002010BDC046A444FF1F7E
:103710005936FF1FF0B5040085B003920291FEF701
:10372000F1F8882263035B0B52051A438023DB0503
:103730009D6A8023274F0092BA68002601901B03E0
:103740009A420CD9F82326001B041E401C4206D0C6
:103750008022214B52025E6219680A431A60002DD2
:103760000BD100F06DFB02221C4B1A608023DB059D
:103770005A62013A9A6200F0CBFC0023039A93420A
:1037800020D1002D0AD100F05BFB144B03221D60F9
:103790008023DB055A629D6200F0BAFC8023BA6880
:1037A0001B039A4208D9002E06D000220A4B0C496E
:1037B0005A621A680A401A600198FEF7B7F80020AA
:1037C00005B0F0BD009A0299D2181278CA5401339C
:1037D000D4E7C0469844FF1F00C8004000C0004026
:1037E000FFFFFEFFF0B587B0029103920400FEF7E1
:1037F00089F8019000F024FB802302250122234E4A
:10380000DB0535605D629A6200F082FC204F3B6808
:103810002B42FCD120230493049B5A1E0492002BBC
:10382000FAD11C4D2B68002BFCDA0120FFF74EFE6D
:10383000002802D0112007B0F0BD2000039A0299A1
:1038400000F066FB022304003A681A42FCD12023F0
:103850000593059B5A1E0592002BFAD12B68002B6D
:10386000FCDA0120FFF732FE051EE3D100F0E8FA92
:1038700080230322DB0535605A629D6200F048FC1C
:103880000198FEF753F8E0B2D5E7C04600C000400B
:1038900090C8004000C80040F0B5802687B0040002
:1038A000FEF730F8F605B36A02250393029000F0A4
:1038B000C7FA0123244F3D607562B36200F028FC13
:1038C000224E33682B42FCD120230493049B5A1EC2
:1038D0000492002BFAD11E4D2B68002BFCDA01203C
:1038E000FFF7F4FD002802D0112007B0F0BD200042
:1038F00000F0F6FB0223019032681A42FCD120232B
:103900000593059B5A1E0592002BFAD12B68002BBC
:10391000FCDA0320FFF7DAFD041EE5D100F090FA8F
:1039200080230322DB053C605A629C6200F0F0FBBE
:10393000039B002B01D1FFF703FE0298FDF7F6FF72
:103940006B461879D1E7C04600C0004090C80040DF
:1039500000C8004007B5000201910422000A01A935
:10396000FFF740FF0EBD000073B5050005240B4AAC
:10397000A3005B429B1819686B46DE1D300000F007
:1039800097FA022804D133782B55013CEFD276BD4B
:10399000052CFCD00128FAD10230F8E714090011F7
:1039A0001F2807D8012380228340D20591680B434A
:1039B000936070473F2808D8012380222038834035
:1039C000D20551690B435361F3E75F28F1D8012316
:1039D000802240388340D205116A0B431362E8E726
:1039E0001F2807D8012280218240C9058B68934394
:1039F0008B6070473F2808D8012280212038824000
:103A0000C9054B6993434B61F3E75F28F1D8012265
:103A1000802140388240C9050B6A93430B62E8E776
:103A20001F2810D880230200DB05153A1968012AE7
:103A300006D820229143196019680A431A6070471A
:103A400001228240F6E73F2811D880230200DB05DF
:103A5000353AD968032A06D810229143D960D9682B
:103A60000A43DA60EBE7012220388240F5E75F285D
:103A7000E5D842238022181A413B8340D205516A7F
:103A800099435162516A0B435362D8E710B5040061
:103A9000012813D1A022184992050B685B015B092C
:103AA00013430B60154B164A19681140154A0A4317
:103AB0001A60402219680A431A6010BD0028FCD120
:103AC00001000A2000F01CF921000B2000F018F979
:103AD000C0220A4B920019680A4340211A601A68F2
:103AE0008A431A60B022044912060B685B015B0925
:103AF00013430B60E1E7C04614F000401CF00040A7
:103B00007F00FEFF80FD010072B6074A1368013393
:103B100013600422054B1A600023054A13608022BB
:103B2000D2055360FEE7C0467808FF1FC0F0004092
:103B3000C4F00040044B054A1A60054B1A6000228D
:103B4000044B1A607047C046140AFF1F841E000011
:103B5000380AFF1FC4F000400023034A1360034AE1
:103B60001360034A1360704754F0004040F1004076
:103B700044F10040002310B5184C8AB00093019323
:103B80002378012B27D06946012000F0E1F90028B5
:103B900017D1009B12490293019B06AA0393114B74
:103BA00002A81B680493104B1B68059300F070F982
:103BB00010220E4906A800F0DBFA002804D1FF23EA
:103BC000237000200AB010BD0123094A074902A84A
:103BD000237000F05DF90120F4E7C046C865FF1FBF
:103BE00010290011082900110C29001120290011A9
:103BF000CC65FF1F13B501246946012000F0A8F928
:103C0000034B00940193FFF7B5FF200016BDC0469B
:103C1000BB0B000010B5FFF79FFFFFF7EBFF00287D
:103C200002D0024B984710BDFEE7C046E1A200005B
:103C300002B4714649084900095649008E4402BC45
:103C40007047C04602B4714649084900095C490002
:103C50008E4402BC7047C04603B471464908400018
:103C60004900095A49008E4403BC70470000000017
:103C700001B40248844601BC604700BFF53501002D
:103C800001B40248844601BC604700BF2D6C0100AE
:103C900001B40248844601BC604700BF6DF60000D5
:103CA00001B40248844601BC604700BF71B0000007
:103CB00001B40248844601BC604700BF8937010057
:103CC00001B40248844601BC604700BF791201007C
:103CD00001B40248844601BC604700BF090E0000E1
:103CE00001B40248844601BC604700BF1DB4001106
:103CF00001B40248844601BC604700BF090E0000C1
:103D000001B40248844601BC604700BF0DA0001109
:103D100001B40248844601BC604700BFB70E0000F2
:103D200001B40248844601BC604700BF016701003E
:103D300001B40248844601BC604700BFC1F70000DF
:103D400001B40248844601BC604700BFBD0B0100BE
:103D500001B40248844601BC604700BFF9A60000D8
:103D600001B40248844601BC604700BFDD0A01007F
:103D700001B40248844601BC604700BFD9B00000CE
:103D800001B40248844601BC604700BFD54401002D
:103D900001B40248844601BC604700BF7997000027
:103DA00001B40248844601BC604700BFCD0C01004D
:103DB00001B40248844601BC604700BF691101009C
:103DC00001B40248844601BC604700BF8D820000F8
:103DD00001B40248844601BC604700BFE9270000E7
:103DE00001B40248844601BC604700BF016C010079
:103DF00001B40248844601BC604700BFC1A5000071
:103E000001B40248844601BC604700BF6D0B01004D
:103E100001B40248844601BC604700BF8D11010017
:103E200001B40248844601BC604700BFA9D8000025
:103E300001B40248844601BC604700BFED68010040
:103E400001B40248844601BC604700BF75A9000068
:103E500001B40248844601BC604700BFADAE00001B
:103E600001B40248844601BC604700BFC11501008F
:103E700001B40248844601BC604700BF3D710100A7
:103E800001B40248844601BC604700BF85C1000000
:103E900001B40248844601BC604700BFDD3F00001A
:103EA00001B40248844601BC604700BFF9ED000040
:103EB00001B40248844601BC604700BF913800113C
:103EC00001B40248844601BC604700BF01340100D0
:103ED00001B40248844601BC604700BF51B80000ED
:103EE00001B40248844601BC604700BFC95C0100C0
:103EF00001B40248844601BC604700BFC9A9000064
:103F000001B40248844601BC604700BFBD5C0100AB
:103F100001B40248844601BC604700BF95730100AC
:103F200001B40248844601BC604700BFE90B0100B0
:103F300001B40248844601BC604700BF0934010057
:103F400001B40248844601BC604700BFF90D01007E
:103F500001B40248844601BC604700BFE1AC0000E8
:103F600001B40248844601BC604700BF053401002B
:103F700001B40248844601BC604700BF0D520100F5
:103F800001B40248844601BC604700BF21440000E0
:103F900001B40248844601BC604700BF01890000AB
:103FA00001B40248844601BC604700BF1907010004
:103FB00001B40248844601BC604700BF116E000096
:103FC00001B40248844601BC604700BFE51201000D
:103FD00001B40248844601BC604700BF496D01003E
:103FE00001B40248844601BC604700BFEDA5000053
:103FF00001B40248844601BC604700BF01D70000FD
:1040000001B40248844601BC604700BF75F8000057
:1040100001B40248844601BC604700BFB3520100AE
:1040200001B40248844601BC604700BF85520100CC
:1040300001B40248844601BC604700BFF935010065
:1040400001B40248844601BC604700BF53B9000078
:1040500001B40248844601BC604700BFE917010073
:1040600001B40248844601BC604700BF89140100C6
:1040700001B40248844601BC604700BFDD0C01006A
:1040800001B40248844601BC604700BF85120100AC
:1040900001B40248844601BC604700BF613701009B
:1040A00001B40248844601BC604700BF156B0100A3
:1040B00001B40248844601BC604700BFC1660100EC
:1040C00001B40248844601BC604700BF19FA0000F1
:1040D00001B40248844601BC604700BFA1AF0000A4
:1040E00001B40248844601BC604700BFA96F0100CB
:1040F00001B40248844601BC604700BF4DF900008E
:1041000001B40248844601BC604700BFE9F60000E4
:1041100001B40248844601BC604700BF9DA900006D
:1041200001B40248844601BC604700BFED6B01004A
:1041300001B40248844601BC604700BFE9D40000D6
:1041400001B40248844601BC604700BF21A90000B9
:1041500001B40248844601BC604700BF9D6A00006C
:1041600001B40248844601BC604700BF5976010093
:1041700001B40248844601BC604700BFCD4C010039
:1041800001B40248844601BC604700BFE94C01000D
:1041900001B40248844601BC604700BF8944000066
:1041A00001B40248844601BC604700BF8B52010045
:1041B00001B40248844601BC604700BFC56D0100E0
:1041C000020000005ABD00110100000010BB0011E8
:1041D0000200000056BD0011010000000042FF1F58
:1041E0000200000018BB0011010000000863FF1F5F
:1041F0000200000054BD0011030000007C62FF1F9C
:1042000012000000020000005ABD00110100000071
:1042100058BB00110200000056BD00110100000053
:1042200055BB00110200000062BB0011030000003A
:10423000B762FF1F0200000054BD00110300000020
:10424000CC62FF1F0200000056BD001101000000FB
:1042500054BB00110200000060BB0011030000000D
:104260008D62FF1F0200000054BD0011030000001A
:10427000AE62FF1F020000005ABD001101000000E5
:1042800098BB00110200000056BD001101000000A3
:104290004943FF1F02000000AABB001101000000FB
:1042A00093BB00110200000056BD00110100000088
:1042B0004843FF1F02000000A8BB001101000000DE
:1042C000D462FF1F0200000056BD00110100000073
:1042D0004743FF1F02000000A6BB001101000000C1
:1042E00083BB00110200000056BD00110100000058
:1042F0004643FF1F02000000A4BB001101000000A4
:104300007EBB00110200000056BD0011010000003C
:104310004543FF1F02000000A2BB00110100000086
:1043200079BB00110200000056BD00110100000021
:104330004443FF1F02000000A0BB00110100000069
:1043400074BB00110202020202020000914A001135
:104350008F4A0011ECBB0011900118001800FFFFFC
:104360000701020304050602010600000000000028
:10437000000000000000000000000000000000003D
:104380000000000000000300020000005ABD001100
:10439000010000006CBC00110200000056BD0011BD
:1043A00001000000F843FF1F0200000076BC00116E
:1043B000010000000263FF1F0200000054BD001155
:1043C000030000007065FF1F0200000056BD0011D1
:1043D00001000000F843FF1F0200000074BC001140
:1043E000010000000463FF1F0200000054BD001123
:1043F000030000006865FF1F12A6A6A600000000CB
:104400000001000000000111FFFF00005048593674
:10441000000000000000000001000000FDBB0011D2
:104420000B000500F7000000B40000280028002859
:104430003075A000A000A000A00000080008E00166
:10444000F0001000100010001000100010005000CC
:104450005000500010001000D007000000000000C5
:104460000F0001000500307507001000010081FFFA
:1044700000000000FF000000E5710011ED6F001169
:104480007D6D0011FFFF0100FF000000019C001185
:104490007D990011959800110000000000000000B7
:1044A00000000800040000003B0001085902E00180
:1044B00088212800FF000000020000005ABD001102
:1044C0000100000020BE00110200000056BD0011D6
:1044D000010000003545FF1F0200000052BD001121
:1044E000010000008469FF1F0200000056BD00119A
:1044F000010000003445FF1F0200000050BD001104
:10450000010000003245FF1F0200000056BD0011EF
:10451000010000003045FF1F020000004EBD0011E9
:10452000010000002845FF1F18001800000090013E
:104530000200000302020000020000005ABD001148
:104540000100000034BE00110200000056BD001141
:10455000010000007845FF1F020000004CBD001163
:1045600000000000000000000200000054BD001127
:0A45700003000000A469FF1F20FFF4
:040000051FFF184180
:00000001FF
